:100000000C9462490C9481490C9481490C94814967
:100010000C9481490C946A4D0C94CE4D0C94324E44
:100020000C94454E0C9481490C949C4C0C94814941
:100030000C9481490C9481490C9481490C94814918
:100040000C9481490C9481490C9481490C94814908
:100050000C9481490C9481490C9481490C948149F8
:100060000C9481490C9481490C9481490C948149E8
:100070000C9481490C9481490C9481490C948149D8
:100080000C9481490C9481490C9481497F7F7F7F36
:100090007F7F7F7F7F7F7F7F7F7F7F7F7F7F7F7F70
:1000A0007F7F7F7F7F7F070007047F7F7F7F7F7F4A
:1000B000077F7F7F7F7F057F047F7F7F7F7F7F7FBD
:1000C0000F7F0E7F067F0D7F0C7F7F7F7F7F1F7FDF
:1000D000177F167F157F1C7F147F7F7F7F7F007FB8
:1000E000277F1E7F257F1D7F247F7F7F7F7F187F57
:1000F000207F217F267F227F237F7F7F7F7F7F7FDF
:10010000107F197F1A7F1B7F137F7F7F7F7F0818E7
:10011000117F127F0A7F037F0B7F7F7F7F7F081015
:10012000081F097F080F027F08197F7F7F7F7F7F6D
:1001300008027F7F081308117F7F7F7F070C087FED
:10014000017F080B7F7F08077F7F7F7F7F7F080706
:100150007F7F7F7F7F7F7F7F07037F7F7F7F047F1E
:100160007F7F1C7F1B7F7F7F7F7F7F7F037F0810C8
:100170000C7F247F237F137F7A7F7F7F7F7F08110F
:10018000147F081908200B7F7F7F7F7F7F7F7F7F11
:100190007F7F7F7F7F7F7F7F7F7F7F7F7F7F7F7F6F
:1001A0007F7F7F7F7F7F7F7F7F7F7F7F7F7F7F7F5F
:1001B0007F7F7F7F7F7F7F7F7F7F7F7F7F7F7F7F4F
:1001C0007F7F7F7F7F7F7F7F7F7F7F7F7F7F7F7F3F
:1001D0007F7F7F7F7F7F7F7F7F7F7F7F7F7F7F7F2F
:1001E0007F7F7F7F7F7F7F7F7F7F7F7F7F7F7F7F1F
:1001F0007F7F7F7F7F7F7F7F7F7F7F7F7F7F7F7F0F
:100200007F7F7F7F7F7F7F7F7F7F7F7F7F7F7F7FFE
:100210007F7F7F7F7F7F7F7F7F7F7F7F7F7F7F7FEE
:1002200008277F7F7F7F7F7F7F7F7F7F7F7F7F7FAD
:100230007F7F7F7F7F7F7F7F7F7F7F7F7F7F7F7FCE
:10024000017F7F7F7F7F7F7F7F7F7F7F7F7F7F7F3C
:100250007F7F7F7F7F7F7F7F7F7F7F7F7F7F08158F
:100260007F7F072408057F7F7F7F7F7F080D070B37
:1002700007237F7F0713071B7A7F7F7F7F7F7F7F27
:10028000071C7F7F7F7F07147F7F7F7FFF1F627F39
:10029000C23C006088FFFFA0089001324006C8C63B
:1002A0000019FF03050A4414812241CF068AF32076
:1002B0000365FBA00C94290034FF7FED81325006CA
:1002C000CA54CC1928E0C0D3F3A9C688009E98D39D
:1002D00064800C7FB9A0FB0014C00287580BF86043
:1002E000012C800460430ACD0270F34032F305A074
:1002F000E6180CE4B312CCE050DBC008286D17E020
:100300005026D334D3B00416E1B998FC3164FF1001
:100310000C0240667AEA4004080C01206D0480A2B9
:10032000E008CA60E4D8F9304866FF98FFFC205C1A
:100330004D986C7A8E8051FC8BCD36A8259ECF4E81
:10034000238202D0340AB923160DB6140A514E5135
:10035000B3FB02882FF18DE346D13C08D13244042F
:10036000B22F0D21939502D203A0A27FC29215FA5B
:10037000201412EC43D307C005256608F4E90003F6
:10038000EE9921DD34DEC81228F388E131D5670803
:1003900068C209D2486EF344FF2E44B4A43BC74060
:1003A000FAC17BA5EF03C6FBCBCA830AFFD36078F3
:1003B0009C0C68FDDAF70CAE9A025A333034E882AE
:1003C00010686260CA3006311B1B0D29F778FC816A
:1003D0003F77C0F98021047BB71020F06081802234
:1003E00060B00740088BF008469C79B0E18C1BADEB
:1003F000B4093E3C80883DD48081FB44D2B008F6ED
:10040000101F936001F9408245B0009FF24418111B
:1004100089F3599FE767BBC006C01833F76B05A186
:100420003148F30438FE463C18C8F280DD1F1840FE
:1004300003E001C53C88F032001EC03A78400FED61
:10044000C3109AB3D2E04124F0D8F3FF9714D3FD40
:100450006E0FB9E7FE8001A330735F978C738EF344
:1004600085016152B69C08CF00658DE097F481AD9F
:10047000F918475DC6D8FBC280457FF3F70203FB3E
:10048000483C11310522221905097E6804C53F4503
:1004900006B6D034B36F665808FEB941340ED0FAB0
:1004A000FF019842FA024113094425ABBED02C95B6
:1004B0008AC36C65112818BD89A0796BCDFCB4FD89
:1004C000B7B698100352E102CDE386636A18F4943C
:1004D00080F77788FB401CD616A303A9DA03F02027
:1004E00033B33E85D9586471AF9FC26816D3A380D9
:1004F00077FDA821172671B00B0151037694C096A1
:1005000069A1E6197FAC981049E94CAF214D987369
:100510001944C069C9A9A498815449120AB381A297
:1005200058619FCB81E0131E15BE2C82091F01E983
:10053000FF5EDF9508F2ED750118DEC5BC0C19BC35
:10054000981B1216B3E027F87F480BDF5E3D08F0DA
:10055000FC84BB41D6A520DC3079F3766460C57E8F
:1005600099C4CBEAEE88F65161FFD3D04B087D8861
:10057000A0404177A9011043F3F821661EB30C6334
:100580001F2EA6201901340660FC0608047FF41013
:100590004402404308160D64F6245F17FD6496BCC0
:1005A0006C0CB5226C644003DE7F3081214804026C
:1005B00070FC71C4B72F300CFC5340B1DAF5FF0367
:1005C00088B50020E8D617A585E7E60D069AE0FE77
:1005D000FF626D19E201AA1903CBFDBF581374E63F
:1005E00088FDC2A421A141F4C29723F812B3B80434
:1005F000DFD6591176AFB1012328B32F873082841B
:10060000809C408E50FB5944FA7A94910682207265
:10061000E03022CE9BF223622FF69312ADF889913F
:10062000AAEC20E5AA44A7C935C17EFD488221B0C5
:1006300008F06E491CBDEF20F306C00318AFA4CC30
:10064000013DF3909AFDF3781618092DEB98C03B05
:100650009A3007E0E730D0FD80CA41202DC8C87924
:100660008340564BA910C0664B61FD278030365938
:1006700066415F8CBD01B218BF10D39881C6F0856A
:10068000F911707C4048690F51C001E52C39604F69
:10069000B717826D499BA2FC2FEFFFCCC20110025D
:1006A00058FF20B544C9C8CEED2420227F4840D849
:1006B000230A9FA8EEA419CEEB16FD98405FBB1B42
:1006C000B8FC71889DE62F7F9BB825A585CD8AB3A0
:1006D000FF8441C97080FBD33BC818C0BF2E807611
:1006E000E4CEA0B30B033481C67AB194345861C010
:1006F0004138CBE0FAACFDA980AC42CAB801F3DEC8
:100700007F5004654A52AC896D870E6797C042CC12
:1007100011E4848EE780043F09EBF9033130AE2108
:10072000783D18052340748CB1971166165C58C843
:100730008FEF7F0433663B911876BC2D8C8081B09F
:10074000EDAEFDE033C81EF8C08318200FC80CFFC3
:100750006C988078B51844B7EFB240CBC873FF7F70
:100760007C980FE4010C201AFAEBBECDA0FE8CE2BF
:1007700066CBC8C5F543A96EAA588403FC4ECC3499
:1007800066E530417230FB6FD031F87F3203801460
:100790008480A6CBF5980399F5CCF5F9BB6C843B26
:1007A00048172F7D4F342128FEAE66C88255680257
:1007B000E6300482FF5998809C30D9500219C8DC79
:1007C0004001BF6779986CE9DBFDF96DF72F721076
:1007D000E23033F7F75A106EC7469E27BA41046DD0
:1007E000EE70F8B3C8C00260FCDF0E20E798F9187D
:1007F000907EB5C25CCD886A621FC9AE58A5BFBCE9
:1008000020B673C84050B3444620BE98B421F5E5E5
:1008100084AA2144D5BB0A5FB0B31472FBFE4530F5
:10082000014DB302FF65C812D6B88357C0CD7FD043
:10083000C6DF32CA1360DD594F0ABE982D467F735A
:100840002365ED4F7B988411C73108B6FDCDC8C82C
:10085000703D577E6907FE4330797F2C3004CE957A
:10086000FDE0D0961CE0B2013D980477B898E00115
:100870003C3A68FAF3F2BC5BEF350BFD87A2C2C3CA
:1008800066CAFD98409DDBA5033FCB98B82A69F85E
:100890005741E6C84831B30137191012EFDC5060F8
:1008A00065E8FCB7D533F8D7B398F898A4E6ACFB65
:1008B000BFF7CE98E530827DB97C1DAEFE3561F57F
:1008C00098019FC363E4026FC289D5CAF798027486
:1008D000FB67F030D9A7200620C66E3F92B77BBCDD
:1008E00002B2C8FF579818DA891A537998AFAC99B1
:1008F00002D5AB81B90E1C5D096DCA3040EEE2F83D
:10090000FC8F26F198F259C85F68EB102054D698F6
:1009100011865277D232F080CB370CE130FDFF24C4
:100920000A5BFB803130095E98899823E901102C1D
:10093000960AD320A1DE0B60B1141FBD3276466546
:100940006A6206222769274C840581B0A9AFFB396A
:10095000DFF21EACC4EEC80F245716B0F72283781E
:10096000F9989BB743FA9807D81851C6F37A9810AC
:10097000FF7E98813C0850F880FF3F988530C36D1A
:10098000CB7564FE9867ED509FA2FCC68DF3FC9872
:100990009BB939FD47B3209804F40340444CE01B55
:1009A00022886FED983004B7D98766C069F3AFB07D
:1009B0009834226BF8CDDF32C8F63A2104FE6BD0B2
:1009C0004003EB7F56951168B3AFDFDCCC02BF79F3
:1009D000F2B7AB9848CB67797280FBF864F6348441
:1009E000DBE53E0C8E2C1980EFCEB504390850BAE9
:1009F00017D1F1D06DA76C9E81615E8D67FC32DBF3
:100A00008107723060CBC8C81F2808E8FDA4BD214B
:100A1000688078D024E4DE2012EF68AB676E960819
:100A200051DD668967C809261378F9DF0444D317B6
:100A3000B48B39F92CC8CA21B5A6DE9060BD61051A
:100A4000D90108AD1290011C9C42DA23027A98C6A3
:100A5000BF32092E1ED162F67F2B3010DAEF0EC89E
:100A6000FFD90F60815F69D3F0403978105EB8829A
:100A70000CC47D98017F19303E984319C66847B968
:100A80007998A7EE8010F398B704046DF2EFE6585A
:100A9000C4B2FF03CBF398FDE5108E0880B3D622D5
:100AA000A0D618B8B307093002B8A0B31BC3B3333C
:100AB00085B2ED9EB34778FB4B89943C7FFB204485
:100AC000A37271B8301BB3C892D724D4C94299918C
:100AD0009624F37919FA2DA342BF2F8B30C8C5C2D3
:100AE000268CFCF2A53CEAD5DF56388162BB10CCDF
:100AF000D3A7CCD0E74B3008709BFEAB0C6F6E33A6
:100B0000400F3FF6F9CC80188E6247CE7E8C20F2E3
:100B10009032D1BD33445E98CB90FEC2CF8D69E553
:100B20002D04E110B9C2AD08D21101C622CE57661C
:100B300044AD98108C0C955F2C70300C7BFEDDF072
:100B400030B83A5833632440B504E85B5E886012DD
:100B50008C04508EE6D74D7E577E8C7130CB690B5E
:100B6000BD989147F31C81E7CF8205FB49F960BB33
:100B7000803DC8201EC8DC30F060400C902B34C98A
:100B800098740FFBE4010C20075F3553ED5428D90E
:100B9000A88AF4CBF6980608EF9F22F33D10F8FDE3
:100BA0008F80304A9B202EF0DD0682AB35C197073F
:100BB0006178C57DA005A2BBD8D55E0C776C17C047
:100BC000FF0098D3D898B1F94194B3BE060890E0DD
:100BD0004CBB491012DC39086014C9E0053E3A6587
:100BE000EAA7849BC026C135B32070B3C17990D8E1
:100BF00068FFCE9941FAAF637A083BAC50F9FC78B4
:100C0000FFCB88087738F3CEF59828FE4B6282D365
:100C1000FFB6E3C121FF98D8FF28D1669CD1638B32
:100C2000399018FACC33DE0CEFFFD9CC01CB66FE3D
:100C300055E202A75A87FDECAF6CD30457F66E025B
:100C4000AB95044DB52103C6F088FE8D5ECFB1345F
:100C500093FB9D143C6ABEDFEC22A2B16CB930FD5F
:100C600057E1F930C7FBCC18FFCDDDC095B2FDA828
:100C70000463BE7B66ACF19811FCE596A6D8E6B39A
:100C8000FBDF617EDBE9B5FF28FE96CF34FFB310B2
:100C90004FF8DBEA121B67EB18125B190419C1D974
:100CA0009263CD8CF8F98FFEF320C27FDECBB8665D
:100CB000A501468012FAFD1059F7E66A721E20DC83
:100CC000C03B754A207FAA70FA78E0477947FEC892
:100CD0001610C77CECFF0823CC770D211008347D5B
:100CE00088FA6E8D0890A6C26F0B0A04261D0C258B
:100CF000CBD2189E9F8130A008CE5CB6C047ED5481
:100D000002503F42087286D07DD00A4003602766B9
:100D100068B335058206B79150EBE4C048D936B0C8
:100D2000201CB681313A1719012A048E20136FDA7C
:100D3000B256AFEA08650448FBC0B9408FFD91FD8B
:100D40007A631FAEE8E0F880E0BECC22F9CC060161
:100D50008898D7C7ADDE808544C6FF3AD8DCF99FB6
:100D60009879F79938E3CF744146FA27D6643FD68D
:100D7000C5287ED9D0FBAB42081958CC48EB4D387A
:100D8000FB6DF6DB7FDBF8929CF501C7BAB5F6FF89
:100D90001CFACFFBF30D90FF0136D8FF1B9BC3ADB0
:100DA0008008BFF1D06C66B3407F90806181A76EF0
:100DB000E308CC3054D85DFCD82EFD42B5BC10FB06
:100DC000C20E6C5D98FC7BECAA296C0580FEEE30AF
:100DD0001DD519402BC6ECCCA55304EBF8021BDA49
:100DE00013CBDD37AD54D6808D4FD8CC7FFD7798AF
:100DF000FE8C99E3FA11636419D8B1FA932D0B7E36
:100E0000B1BAFECFE55980987146E613FA94FD33E6
:100E100029C64071B486EBFFF07619C401C90A0FE8
:100E2000C47EDAC7FC6FBA64C7790F80613FC9AD71
:100E300021B362E6E43EAFB320B5E550B1FBF34029
:100E400030AF8C055D3AC0B7FBD23E2DC83C599DF2
:100E5000132FD69F0439FB2A4076E418FA588CCF1A
:100E6000CB94B20A5DFF08D4FA925134A922C1B0E2
:100E700008DF7D8BB0FA88B7EDEE81BFDE107A48CF
:100E800040E3F23884E1E22E1512CFF528F3C6FED6
:100E9000E1D13E58BDFEC614592E593244E5CFAFBC
:100EA00020D8DA01A23780D90601A340F27FDA31D7
:100EB0002138874DFD40F310DD34170284FB0143D8
:100EC000416861BF0F304769F397C0A066F66D189F
:100ED0009AEB30150D89819A19F64C26BFD1808284
:100EE000041AA7FAE60578FA074885C82010AFDF8C
:100EF000024AC051209E01BCD0028A8106DE0877DA
:100F0000B350441CCC7E808445BF9901681ECD0639
:100F100086240106E614A462EAFFB7FDF5CD10842D
:100F20009D28BC112B8DA74C49FD2FFCD2D802A4C3
:100F300082E3AF11FB8571113D2393B24652358098
:100F4000F47904A466BBFE0648D5363FBBE80450DE
:100F5000450C4BB6D87C475764D80DFEED4C40BCD1
:100F60006EC4FD7378623AFCB10225C120843A1345
:100F7000DB58F91A30AD2D0CCC29FE37CF31476E36
:100F8000EC8DD8FE637B0D80201C3314DB5938FFB9
:100F900055970286FA1564348D98FF9E639BEA612B
:100FA00046B4E981FE306227BFF5159FFB7D081C22
:100FB0006FA498FBF992D6792488F2D920D5EC1049
:100FC000634645AD6F08F9C6F639B7FA83706339E1
:100FD0007B6EB3B1FB539414F3941C4DFF3866023F
:100FE000845A3363C76BFFDE88FDE0A011247920AB
:100FF00012009AF4F84882800408A23C0E04092DDD
:1010000041308A37A120D0FEBD02D3967AD089EB39
:10101000894A8184C0AEFA0EF7F39FD23A80B9C7ED
:10102000F97CC4657E14C08EA73B83FC8858F98088
:10103000CBBB906590F260E203AEDEB106DD4DA55C
:1010400082018A66B7C0858CC61EBF7C46D0BEEFC3
:101050001F10F80344B04A53286F0C40245ED3227B
:101060006626A90F28C53DF2C0699B984CFE97DF04
:101070008E27490DF9B37CA2264A7F66848C8011A5
:1010800030014643E45C02CB1140F3136966060865
:101090009223AD61BDEAB348B998198CE78489B051
:1010A000BFF9E0FE013CA007F1801EB8712F0FE2EE
:1010B000819A38F301481903F3BBE24113576607DD
:1010C000D067E03D0F02C8F33468C601C638B92CBA
:1010D00008F8FB805030A60646189A0B400C14F313
:1010E00086DB5FC2F610088481286647FCFDA27D7E
:1010F0008C11D3C6FC9D4CC6B0FC0C11B223B3249A
:1011000082106F5A025AB31626D3048905C6D6B385
:101110008C8DF3821ACCF82484F5C61198FCE1DF9B
:1011200044AFD2AFCBD0BB80BE482401DF92E014E5
:10113000EC4941B6109301E07342C94008D3FC4723
:1011400019FBDB8848AD8408B12EC8F8D7C976539F
:10115000407F8B900C7E37E2F1E52D64846A42ADCE
:101160002ACAEE320220D3B920E8FF6ECA30909A24
:10117000E9F41928EAC9E5E918BED9DEBA63A3443F
:10118000FCD4E003D36EDCA2032AF10CADF4F9A881
:10119000091153BB223B0C4401D382049C087A669C
:1011A00081C4F7AA1678E03B816795182002B42124
:1011B000EEC3E9FF60E6B164260119680B3C214CDF
:1011C00002ED5906467E5FC4BF7F80A189B3E00669
:1011D0001072C1044CAB8825F3007A42207AC6B065
:1011E0000849FDF7988807F0F8001EC00379750FCD
:1011F000CCB9800712F3F166E667F4B098EDC4034A
:1012000009D302ED5A400F7EA990C6388876132C78
:1012100025F85F2C01DE98DF0803F798FA9808C5D7
:101220008F19FB6CDDFC22400CAFE6EC18EA60D1B4
:10123000C6A8E1FA8041611006FE08190103601496
:10124000F5ED427EF901C536D8F0B3A9E005F613F5
:1012500060020DBD643EF30320082CE71988FE30C0
:10126000132441C42010CA12497079E59004918674
:10127000E07FB5782120D6507FCF7FB0440204BBF9
:1012800012ED40F5E440CF2068FBA049840F98F8A8
:101290005BFB5E8F72EB60CDD919F362BDFE2E3819
:1012A00032F87930617E798820C8F8469F21FDC0E8
:1012B0004010C8449D8F7AE918DBF6CC1023ACF1BE
:1012C0000424DDE988B695ABB30683CD7080402851
:1012D0003F50FE0C0530224D9418410AECA3FE0A43
:1012E0004001D3E0CC7681103069B5FED2CB4610F8
:1012F00030B9304D15EBB348D203019C3F0562F87D
:101300000F083227A3F68910EB2360448530E92EBD
:10131000B39870D94880094667F5643DB3C0029020
:101320000471307DAEEAB318EF68118C08CB402011
:10133000C9B930907FAF9883E6300C90EF2298D8EF
:101340006CF3413CFF579841BB98F4401EF830F3D2
:10135000EE8BC6EB4F9F301C0848FE04E440302063
:101360000957F591707D12F3D7BD640C88819E19E1
:101370007FA085C13435D3FDCC18FD2D27C64B2168
:10138000FC212667810646982037E08406ED940408
:10139000694673E00530B30A95B311F3DEC058A275
:1013A00008B3F3A598B3041B305017BF5E11321079
:1013B00098FB2011F9C8C59248AF68AC54C9C82041
:1013C000628743D96809B1821EFD16801410221A63
:1013D000DF338D21042ED3F857F203C6FE6B30B4F1
:1013E000F8E340B7E19BE15CB36E79460C71B3BEA4
:1013F000C35676E8E401E0D7C898CA73B8FC40EE5B
:1014000090774EDEB96040FFA3F6D356B00108C412
:101410007C995AE3E7C80C486D9DC60170A7293036
:10142000C819B14E53889042B4FCF5CF141E89C739
:10143000EC81010553973082E7C8282045B8D58450
:10144000CB7B684EE23583FD7C09204026047899E9
:101450005F0B62128C80CB49B0F25EFDFE488809BA
:1014600030049DFA7F417EB34208980423607DAF2B
:1014700090813002DE1ECD0308198C6CF61F69FFC7
:101480006041AC3CBBF58B6ADA98E401E53004A618
:1014900040F5ECE0013D4F9130B05DCD03400FFED3
:1014A0005E7F2D30707830B3C8315DA15A9169E507
:1014B00098E1A51B65F57998897CCB4B80FC980554
:1014C00082DBF67EA5EF62C6CD6621F8A6457B726B
:1014D000E084DB36C81899F55C23623DB1FB21C17D
:1014E000049802658646CD862268D9BB81B048BF84
:1014F000FD3CC8120842A68CE104902DC07EAD418F
:10150000B8523D0D7D9F897B98041443AC3611A2DF
:101510002DE0FA2AF0DB906A7F8121080402D0B521
:10152000FF2D41378FE350CB7F6C69578D30F2D15F
:10153000DCED870CA90110D678F84CC850A0DE531A
:10154000C89B776B8E324DEC7836C4FC9838456E6C
:1015500016C05E02557EA6EA0AFC1C0798FEA8C7C4
:1015600091905C12AF502FC53C2ECFDF3B89B0105D
:101570003C1AFE147D8BF5AF80F57F044612D757D9
:101580006F1C8884F3942082FCB7315F7F9C249A7F
:101590000B600F8C825130FE0146C4041805236B8A
:1015A000F30C8CF843B21701B30428F3C0232004D2
:1015B00038443CE046C2220905A5FE11888021304E
:1015C00006A8B830BD98B1EE001ED0E2307BF3A083
:1015D00007F0804C96BB3629EB98F4BDA5597FA245
:1015E0009880BF903018F20762F3BF3284BF412564
:1015F000C85FB7D112F3AF172399CBFA156DCD3071
:101600002040ECE006C4BBF3E20C13F31F4195FF4E
:10161000469DC8C082B8C0DA39C83DB32C8411B227
:101620008967C810C0B942E002F0889051B02B40E1
:101630008123C701F3140C8409C620B4FEF0987905
:101640001A405A15FC30D724020A30F7F1C5F1626E
:101650005F7F818088FD0240120108813AF390107B
:10166000D4ED3B627330A009F68610F8FD669F3911
:10167000C63010AEFF033525C9C866BB606BE53DBB
:1016800077FF40807A98204D266C40E7162DDC06C7
:10169000562C0824B87FAFC002FA1652E024D002BC
:1016A000B930849C81F3C8F8CF6010A2D0481834B8
:1016B0003D60A2779EB8BD8560208E84CF755B802B
:1016C0000902D4BEBAC11309F28188210432ECEEBA
:1016D000738B687A58942062F8F7980A0601F8022A
:1016E00018050B205A4C82FAACF9CDF35F98F648F6
:1016F0008051307AB2489249C8D33513DAAFD64018
:10170000304E35790382802F57892E23FCF3D2FC8B
:10171000A51578DEC5F738A00702723078650CE4AD
:10172000E6897898F9D34006C081D3BB0B9B300380
:10173000305E1F30F30C0848FDBF80D59820FDCCEB
:101740006040A7969893151910087F1930FB9647AB
:10175000D3E8BCAF731B5E23026E2F30EBB579F874
:101760002BE2C6984601136F024BF0B31D4481056E
:101770009EB32DD314B381D3B88CD3B583190D1672
:101780000C7FC8311078F92009D726419698E12DB1
:1017900068BF9130063748407AAD416CE6024B4B4A
:1017A000AFDD6702422271D97F338024A711C603BF
:1017B0000804D78121B0E3D8FBCBA06D8ABCDFCF72
:1017C000906CF68401539777041E265878E0EDACB0
:1017D000034033C04899F8B321502BBF976220F0E3
:1017E00030CB3982FDD6B1022FE598EAF06226D3DC
:1017F000650501D3C5445767C848FAF4840530220B
:10180000A2A002DED701F0500A1421213D9CB105AF
:101810005F1998D213DBD78D245ACFEF8F228143E3
:1018200073FEFC838430E1101601C818477F118CC9
:101830008005B006161D8866C8602C401B813FC815
:10184000989C7FE0C40298109360EB12408432C8E9
:1018500010607CC683201148C69932F718F8E081E1
:1018600064C855C76A66C841B930746BEB98E0111B
:10187000F59841FE9834D301D36479987330E2012E
:10188000872CC8AFFADF1F20CC3D0260069EE5B46E
:1018900040F0E54C63C898E08FD3CCC8C405FA7219
:1018A000402E0F612338FB6049104C0641195C88BB
:1018B00040069C30DE4842B3D80890864BC8E041D1
:1018C000B312DE6202D3E742C004D35320E4080C13
:1018D00084F36F48FA2000AF243F9836D4429C30FE
:1018E00039F41B019F084718E6972030106E9A487C
:1018F000D282E5CD92FEE3D7080A979874F310FEE2
:10190000A07F9FDBF29452BE563A3CF8C8CEF399C2
:101910003C58DB2D1A7D9880ADFA2E591A3006C836
:1019200034C0E43030DAAFD02CB8314FD498C0692D
:1019300045D6AA633017CC0924AC0BA6E911E0FB0D
:10194000C3A204ACC3B5C8CD5D46F9A29008D907BF
:101950004601A683DEE6B950E42230CC9032124D27
:10196000B8360A100BFACE07418811F494207BF8A0
:1019700019C92146B8DC871324FE8C820530021475
:10198000C012DA8CC9C8C596B1E8C671ABF884BC80
:1019900098BFFB238660EF7C981100C2225889F320
:1019A00002FF2882093012A1FBE0AF414598F159AE
:1019B000C8AF3843C5419090F3351EC491C86064E8
:1019C0005B3C6AEF10D4ABB6ADBD9820766D9B1032
:1019D000F3C8C8F303181007F33D3657FF9E985F0E
:1019E000BE6219C8ED81109056B350ADB38881DE48
:1019F000E59D40C303617998D9C8B2023C98068935
:101A0000FC16111201E0C60458B503DEE326C15DE1
:101A100077996E4C252D0CBAB0C9E2737ED31001B4
:101A20001360024C8ED3EC3B1ABBB3DF9805310A2E
:101A300078FE639F026518B3FBFFF8FBA120CF750A
:101A40007F17AF91585094F36719D126E0C7F3FD83
:101A500032A3D3A8FE6880618AFF08CDF2C9CE20E8
:101A6000FA288CA02E3366D7D342B6D3F0FD72D0BD
:101A700042C6D071011B9BBEFDACDAAA6895B3FDCE
:101A8000961B8046D961C6B631FBEE104E65FDFE51
:101A90000493984409B886B1DEA35B73D38FD7FE55
:101AA0007088FF0334B5C33FDECC04D3DE98FF5A01
:101AB0006CD56FF05B98B26701F3147FAEF2B72B71
:101AC0001AE5B3FAF3D828B8C7CCFF65D7B0B3FB93
:101AD0007EF9C2D5B38094F100B019C4FFBEE9CE3F
:101AE000D3E0F8F9CEF298310CCEB1EC92E0FD7F64
:101AF00084B9439A36B101E3AF39ABC87919E5C867
:101B0000C487E4B00883F67A80503BBFC672BF0238
:101B1000EA01F6C7F84048E2044E06BC0C4105A7AE
:101B2000FFA8D320F16CD61055B3021D99E7D1055B
:101B3000C12B729E7D0180B4062F82020AD61060EE
:101B4000711D0D186114B85E6CDF214FBDAE06A08B
:101B5000306D86CB8541FB3514E604486AF4036694
:101B60009D0C19FA16292007029B10894042F000AB
:101B70001208A0762024AA3701CE294452C43F3748
:101B800022B7A2E2405295841C82E4CE14F7D322FD
:101B9000A0F8FA3901D7E8FB1DC756FF209E0C0DAF
:101BA0007DDE8830E4FB282811B9025F4602B48C40
:101BB0009163BEE2B20145F67992D7CB80FBF02C5F
:101BC000DFDFAC6C738DCAFA2FCA6C3518FC95F345
:101BD000419DFB0040165CB788FB67F35828FD6504
:101BE00079038FE97A8E3656E8FA30E2B1B045E9EA
:101BF000029DFBAF0A666258F8DC28C2677E0222AB
:101C0000401CECD31120932D5F6E24E8FC31997FAA
:101C1000D8A008DF1F7B97C2F91EAAEBFBCFE2B367
:101C2000D3EB1ECD39209ACE6BFE8E88F908C930D1
:101C3000DF9C16CDE34A5681C0FFC6B857C25E3658
:101C4000BF6C35D0FA6B2C8E2ED7EDFE08016C9E42
:101C50006DC690152CBD01A62B50FFCFF9A3A6464B
:101C6000E815695437D24002F9678CEAAF40C6FFE5
:101C70007F80620DD850F99E6763EBFF0116FDB1BE
:101C8000A9863A15B1406689B8FBC656CA6033C604
:101C9000832462D8E8FE97ECDD042A3F5EF65409FF
:101CA0006FAC980221F5A2208D23E008BFAE17305B
:101CB000DF9FCF96D54C808936D468FAA6BC131F17
:101CC0001C92CA1ECEF27AD5F34891B649147129F6
:101CD0008C368658FF57D65ECD2BB2108D98C3D761
:101CE000366DE0FF33DB86401ECDBD4498EFDA78D9
:101CF000F9EA9B09D51D105F6B46D88D7E22408B7B
:101D0000AD7702563320AEF90440060650F8FFC8FE
:101D10003644CACE2EDC32BD966F012FED4F8008BF
:101D2000BA2110DFFD9804F980326B0211B900ED81
:101D3000F2ED47EA41868BDB19E081DE1004484072
:101D40009640144FFFCCB9FC60400580C3B436C246
:101D500002C0B9125EA01C28211C821280F6B54573
:101D600001C02266EEA805A07C72811940012809F5
:101D70000DB41C9A862109D512452351FF4F281016
:101D800090011A9C48C1420CF88F79180121E7D4C0
:101D900002614F6609811204621E99CF2B204F30D9
:101DA00003B88F02A09E01D88094811508A693598C
:101DB000F9F0FD7A34018DF4F3FD046FFBD21017B6
:101DC000DD5C80B1E01BC6ABE5C8B91705207A150C
:101DD000DDDAF6100480408ACF0416D31328B22827
:101DE0008FE0DBA53331A7DECCEFEC78FA50E3D5FA
:101DF000C36831DD481608DE4C92042F8A6D8B1CB7
:101E0000FF8DBC8D79D44A120F67996BDD8FB201BB
:101E10009BEF88FD16DBEA13586380DE6B7138D2C6
:101E20004B280DDBCC2D3C52FF186648D522286983
:101E3000EA3902F3E61AE5BF908BE72430FD6C53D4
:101E4000B2087FF82046FC17E46ECDCBA0B340FF6C
:101E500023B002C11C0279C793FCC9F8FA06090D28
:101E6000FF98FF2D11287909117996FEB971469DC9
:101E7000F6CB3FBD2839FDAFECC2064336E9402919
:101E8000FB9904501E0DF823E0D72F1618F9319B4B
:101E900097081CD05AF7089B57B65028F976577FF9
:101EA0004658B808B309FAB1187F3CFACB5AE0ECAF
:101EB00063268BEB685ED1B124FCB398C008DA824C
:101EC00040F5418B9B4B86F5657A7EF9CFF9A4B33B
:101ED000A380A80C9BFF58FBD6F9308CF203089A1C
:101EE000F6FDF034B058F00CEAC20CF38675FFA092
:101EF000A319D0247AF941FFD157D01E8DFAFB22C5
:101F0000CA5937022819FD0F3D26C208D12C025CA0
:101F10003B69501013BAB015B2899BB48C73D30AC5
:101F2000B2F3B893F1B3267F400BBD0F93E00306E5
:101F3000C0BF0396773C27DB9C3075F63C99CD9665
:101F400020FEA29340F3C3FEDCF39399B38001C952
:101F50006386FF6BE020F864BB5A224001C8190F6A
:101F6000F5B3518AACB32883B32D1940B3FB748801
:101F7000D356D5402BEBA50857F340090166FA98D4
:101F8000209BC734FC285959B5FC596679DCFD3EC5
:101F900062BB2C3BEDE0FB28B3EF3298B3E8086658
:101FA0009BAB9793DB5F7998B7D3DCA1F0FE6ECF44
:101FB0004B2241206DC27F5A9840A77744FC5BFDBD
:101FC000652D2B4CBF5F01BC13F958599FA5980490
:101FD00047A7B655B00847E97F09CAF964E8560D26
:101FE0000F02A37306C8B483F3B814F5EF80193B4E
:101FF000DE9895E0B5F632E235F4DFF098181A7DF8
:10200000EC8BF898B366CBE0FBCCF9F825F02177A0
:102010009E98B3EC20080165B32846C577B5988033
:1020200040FB7FFF27E3CDBFE8AC46FE3830F3D955
:10203000490A6AF8BD05FA82363B0825ED9858F83A
:1020400089EAD408CED32A63341AD93A62B1F92F77
:102050006D9806D01BC90C0812F59820BFEFCC0C68
:10206000E3907F7698E8FF0467AD98803F75036B37
:10207000E6452419D1D048799A337FB69828FC5781
:10208000EF324CE1309322BBB431B34E5B3002FAF5
:102090009820C8F598316EE3FEDCDCBE3CD394306A
:1020A000F019BD03851CB1102EEC54F0204FC998D7
:1020B000B3FF65ED2CB944E219D6DBF6D412FF9BD1
:1020C0007F1803AFB69840F84FDB807B98804806B6
:1020D000A3D0D3C53F420862BE98DA78F969AFA2AF
:1020E000DC0DF4E0D0DF3B21B4E3CE66AD66090D34
:1020F000F9BD9834642919A0EF14716697A92510C9
:10210000F36C2FB380F985026F96006919ED865044
:10211000F9A11EFF7F6BFAACC039E566E09641B4C9
:1021200024B3DBE0807DCCFA2864AC01FC9DDC6943
:1021300024C97EB7424880F4DE7627BBE3D0BECC0C
:10214000CFEC0545E0FC23FE3722B8EE3D46CD0935
:1021500044F649D93002DDB1667030064FD77FB6FC
:102160003061F8E30319409B01DC0CB850FC9DC8BA
:1021700031013C89FECC30DFD69804FD1743D3975C
:1021800098B2F975151071B6A109AE5BC8367E48D4
:102190000148ABA3736612FD7F91AAB328F3886F41
:1021A000404B50B943E021B1303E6CD1C0824BD49A
:1021B0009841F1B2FF3F7F082DDD7D8B12DA61037C
:1021C00099DCBA1DBC03D3DFD4980488B722F198F8
:1021D000E7B2FAF295DFCD980CB34FCC98F3FF76C7
:1021E0001970FBCAEA172519FDE0BA43088DDD4DC9
:1021F000534CEFFD59FC403CA6D1B0FA8BB3D6044A
:10220000207EAD62D0D6CB04CBD6482C6696260174
:102210008BAC102FD498F2B36FFD7F820CB7F6AC65
:102220000810BD176C28667E3201C932667BDBB8A8
:1022300064FA9858E2CDF1A519DE06C06D46F32583
:10224000FBD33072F05BE27079A836C3A0FDFD9E2F
:102250005E986BF512C538B7E3E591BED97BF9C836
:10226000622DE6B9FAB6D276B304D8196DDE2356DC
:102270007C01A6C32F9BC84025AAA8796678D2DB2B
:10228000F30AFFE68802AF492EB88617CF33B3FCB6
:10229000988DBBFF17DCB7F85AD30119C77B092DFE
:1022A000A94C896B2DCFD666288BB3A04FB4ACF365
:1022B000987E165E8079CD9FE1985BF51765C8A77B
:1022C000F5CC9028B96D02C27FA89810B03B433975
:1022D00073C3636633C998241064B6DE1BFCFC30FC
:1022E000BD1269B05F7F834205B9A0E009EC308977
:1022F000024B36C8084B66C0246AB3AC11DBC5FC80
:1023000097EA995F1E987B46403C62451DE6CF4F99
:10231000AC98F09E5A30589D66C410B569A662CB41
:10232000468114E17DFF625B964BDE8123322E0BEA
:10233000FDDBDD98082141FB766719B3FE98656ED9
:1023400049016D6EFDB9EA402DBDFB7E42BD0852CC
:1023500040B704EBFE1CF49860EBF7A050AF64DBD1
:102360009635D520678B28CE1B65FF604066CB571E
:10237000FE2328C819D51610B6C05B230875178D23
:10238000FA9878FD9BFBFCFE4CD7F528B9CC0222CD
:1023900020F31993C240B6CECD7B019BE998098802
:1023A00079667A0904BFCCF80DB7BB981060228615
:1023B000698CC001B4BF03AEB332CCCFA96CC5C029
:1023C00018AF5A980402B35E98D938FF1F69B21A41
:1023D0003D98C8D00302DDB20C3204C5B930F072AA
:1023E000DD708BD3F60068BAAF71ED93EB9808D629
:1023F00066814E58E8DFA89860EEE548FB93EB98BD
:102400000A6F51988019EBA60973E21AF398D5194F
:1024100045F7969F66DA9E88F298FB7EBFE742DA20
:1024200050A02C390648B457E01803970530B7F888
:102430003D5314806CE767EDED94E7466625CB309D
:10244000C0CFB3CAD5768E0C088084AC5B47439A64
:102450007B189949C6308BB3D0DB890A206139F4E7
:10246000662DBE108C66DF5998047C30D922FD3F62
:102470007F5E98B401F8BF370AF3308210B502CB03
:102480001351C3DF72E048CAF59802AAB3216DFC6C
:10249000F87D982039EA0319BCA36019FC9888AA32
:1024A000466DC4071BD5900325663046C5579B98DB
:1024B000AC19D88ED817038F375DA0058DF6D902D9
:1024C000A9668DF23071C966B32084D428F3E0F494
:1024D000FC80E0ED0204566E0257525CDB02C4B988
:1024E00030482C196CFFD4B38CC32165FFF8FB0C6A
:1024F0006EFD105FD2B6E380F39B99F3DF32B22812
:102500008CD3E0C638A0FC0C121DFF98FF249E93CC
:102510000590F3672CD1206D66C8B3FBCBCFCCAA56
:10252000205B7B6019F75F1ADB68FE19739D62718F
:1025300093889BBC9AD301736A397F4DEE6AE0A7FA
:102540001BCA9E24B12F4423A4D113316A0384569D
:10255000B1F0FEC47EF9C36FD8CC988FA39840B772
:10256000596E08BD1D62DC6568CFD8A0F825F9E575
:10257000830AB301CECD3420845DB1B1FA1DB31C02
:102580007FF20428A5EBCBFDD440BED1E3E4BFEC41
:10259000AF3053F6CC10265263EB19FE143CB82230
:1025A000C5F2CAC50BE94C15972E1004026AB7DABA
:1025B000048178F07679B8965FAF10329F569FA568
:1025C0004E7D2E0840810923DFA01BF650F7882D91
:1025D000D8042881142DCA54B76A14B725F328B338
:1025E00097B0BCFAB7D9780141F3979E295E596E2E
:1025F000625D637A7A40D37B1724207FADA165A604
:1026000030FABE8221FF30A1D0FF195BB0B802972B
:102610009619042CCD5D7B6FF1DD113397ED7F4C66
:10262000FE8A7AE606FF30BAB563D8B2FCCFBB3774
:102630005258B802B1628B75FE830F6C1780336CF1
:10264000B318FF1B397D20B508FBAF37EC70FEAF28
:102650008B3398CD25F5B280D82010506AB920FC74
:10266000FDB1088EB0307CFBCC0555B30199B66442
:1026700029D6FD37CD13E8FA8DB6940408C6F711B4
:102680007F7F90FD626BE5440D1619FB3CDE62799D
:1026900079629A4DB02887EC7F276C1550FB157C2A
:1026A000E58D308C7C345DB3C8B6E32F9B4B050BB6
:1026B0003749F81D9FC60933B6E93B9DB338FCA9DD
:1026C0006B9E656EAC0D929763995FB1A8FFD87F42
:1026D0000151DB0A0804AED864DC43E64B13FE7FED
:1026E000C8DC668C37AD506401F3B048B7F67CFFA8
:1026F0003FFB47022C8258CEC72DBE589319087A4B
:10270000205B1A8940807A6581C694A320AE7F1928
:102710004F2A458060AA2CFC5C03F5E6010210E616
:10272000509BDE0580929350CD8CEBEC816628782F
:10273000D56A9653EFC2B3306036B0A0AC472005DF
:10274000DAC3887ECCC047E1860297F709F7B5184F
:10275000029442D1A76C8ABC1044F1ACC1E0921043
:102760009034D28F43F30D2F7E69DDD420F8F962C7
:102770005F4EB108CF3516595520CDE930F8BAF57E
:102780000180E33CB747A482818DF3C3D7B72166AC
:10279000FA446EBA387C0220EDFE76B649C73DB9E0
:1027A000146AD8B20850751018AAD31CE36674A432
:1027B00009B46131D1CCB1BD66B3F8FBC25CBC5287
:1027C0009CC77BDF98B2FD7DC0806701C161676CEB
:1027D000FE309ED8FE40E939B90C845AFCA588B970
:1027E000028B2CC64021EE0540FDC67ED5CF58D3C6
:1027F00080E9B3FE4B63992AB110B3032534C8B006
:10280000FA9396CD01117F7FA8FD63AB90146EB053
:102810009E8774DC9019613EEC9408E5960C980351
:10282000D858F8D1698FFD679F9F2E840486C06AAF
:10283000F2FE8D24483402200445B24EAE012490AD
:10284000C49EB892169018060363BEB95DD7CF51E7
:10285000481A4162E708808C4A3442DCA8FC3AB24C
:1028600004423831FF524644FC03E5F741A3CB0450
:1028700001B8400F99B7FC60C96CC03CED604110D5
:10288000769F472582888927B60C4DB040D006C078
:10289000B3DD2D81D5BDE828021B400F9A6C50FF97
:1028A0005BFA0238710CA1050D34FCF0654C43B3A2
:1028B000F085FC16DEC102669D4C173021CE6648BD
:1028C0000B013D0D3FF70A50FC8011B0DA2046B3F2
:1028D000D44C8046219526F8FFD360012C80622FCE
:1028E0006548302040FA81045810080AAF19C00A20
:1028F000C0B71522D064047D5F0898F9E0C1810C4F
:10290000B503F76C0FE801E63C8007BC067EFD7856
:10291000100FE241CF73B4E00138E0F0C3201C7027
:10292000D3D3F33DEE801E380C3810A6CE3C37B81A
:10293000F98028532AD519823BF31006D31960F386
:10294000846207B30ED3732018F6D308404A59F3B4
:102950005FD303C3FAF388CFFE80932212046C196D
:10296000E8492001B352E3B38C58E683B341340203
:10297000845EC0B3392F0530134DF30153FAF70EBF
:1029800002B6E36FE2885FD703F97A84EBBF045F96
:1029900024024C2804846777FC88013CE386C082CB
:1029A000CED410B401A0F66F4898360869E7F72432
:1029B00020C8B7FE3FD6EBC72F29F2E838F75F1BD8
:1029C000630055F8867BF206C06DD6DADEBBDA020C
:1029D00060068FB6F9F561C0B79247DD1EE5DD0FE1
:1029E00019D2D9B7EBC4010CE5C9B0EB16E0F2D4AB
:1029F000BFA003B9027E280F30FD21D8EC41169FFD
:102A00003BFBD7768228F04183CEF5E3A079A5B3CE
:102A1000A12C24B509ED360AE88AB41A32FF57A36F
:102A20001193495F621271967D7FCE6D601480763E
:102A3000A8B00821AFCB0640C204815893FB604484
:102A4000800284872F900910BF60DD1B4198FEDF54
:102A500069BD0719787E79B7880701195E98301922
:102A6000622C3CE4B560090D198BF01CE5D00370B5
:102A7000E0FF802B14B5A41AF7D625D3FEC87DFC41
:102A8000A950C1A0DBFB980240D8301081662B8989
:102A9000408EC935E0FD95101ED3E6DC99FB19B4D4
:102AA000A6FD7221E2FAB3BCC5E1B3F41D88EF5272
:102AB000124080C490B368EF2CE5CAC076338B0512
:102AC00042CDB321C00019CEA106CB8208036F7797
:102AD000981428127230211E0835D9BE0A6AF89F50
:102AE000254C8020C1820343124AEEA0E1EA86F51C
:102AF000489A4062DF56A031040606F9CEDD5D201B
:102B0000B79898AE4A4A9A3726D59906A72D30101D
:102B100009CF190C2C91BEA381AED2FD60D8DF4C39
:102B2000119DE92F0632BD02BB19CDC3B9306045F6
:102B3000FBDE6468FB0493D646BF40B508506612BE
:102B4000FC3B0490B822E1B433F830D7941B1192C7
:102B500086805FF8CC30034143F351F5200288F9B9
:102B6000FA3241F997EC47DEBD5346C004487F3244
:102B700012285CBDB60AFB8A56F809404E761A4800
:102B80001877D501148D50F2027130C99F50FDAEF7
:102B9000F0AE17003DFFB53CF798F1200E017B9891
:102BA00003E0D9413CDD17FCE8010CA00730C0DB95
:102BB000D0776BB181F7ECE2733078405C16F73C6C
:102BC00010C8FB9109B61A73771706C0470D3BF37F
:102BD0000280303B3DD681413013F38983606AEE39
:102BE000BBC28D305B9368FF8BB3D4F588C0BD1436
:102BF000C806F440040805B39B44DAB03BB317841D
:102C000006129A46D418F26D5F6920E898585A0B5C
:102C100064570F85E9D2F8A6802FE0DCEF04D36873
:102C200050E9142477F0DD22016C49FCED71A0110C
:102C3000393043FA0B68140D08FB58B93040FF6275
:102C400068842D28440402DC18FF8805C7CB915303
:102C500059B97679DB9FDB17405E4030806CFB2BE7
:102C60000C884BF4BB7740496610BB7AE570D79D62
:102C700030B020161DDDE873380CEFDA3281713088
:102C800064317C0862A2DD8367270222FB82813BDC
:102C9000F638FD97AB82FE8568E2FB4DF2D0570512
:102CA000DB5DB780EBB1765E89018FA8F111F7AFDC
:102CB0008CDDE840F09BCE2C224C9D6611B2FE2F9D
:102CC000A30A77651360116A8206653920DC7B9858
:102CD0004C02EC093001CFBF32D5B226EC98091076
:102CE000E14980822E2FAAAFBF489814C7806B217C
:102CF00018AF64CAD5FD69717AC541B923F1020ED6
:102D00006B767838E8803C1603676EB1E2F498344D
:102D10000A1CF6A5200F1BF2C8510CF330D3813CDE
:102D2000F4B0FD6679D36D360D0E0620FB1F7708D3
:102D30007D83EDFA643B625EF8CF7780F130C6396F
:102D40009C30DE0361BED708A1DD32F78FFE32145E
:102D5000B21DED74D2281802B3E32C800433FD4B6E
:102D60008032CA06FD78B30A4182538194057F3CC4
:102D700030034082082D0531F9C81AA05F8793C837
:102D800076A0178040DE00D4C41329245D2B6A642A
:102D9000B788F54B057A981087679921A2BF01D1B2
:102DA0009858B88B6842152091C82DFF8B872DC885
:102DB000BA7EDF9B3010A055EF44AAF88251A3469B
:102DC000A805DE6D01D36FDA4030F2983B5DD999EA
:102DD0000350F18F400C778ABDD72EE5A364CE5304
:102DE000D75618C8016BE007F3F680BD1028F6B37C
:102DF000FC83C821A720C02810D0BBFD943016D476
:102E0000AD40AE29BBD1C598A21C9E65360C058B82
:102E1000BB4A5411A5EFF89206EAF76F529010C919
:102E2000BBC402604CFC6FB40D2AFDDC3010A4DC86
:102E3000C162FD898241304026799870BDE13A82B5
:102E400045580A9673C8C40469032B7DEB33F85FB9
:102E5000C088B20984EE4230A0BB90CD9873C87090
:102E6000D7200F0C6AF3F4AE39403020AC60B1AE1D
:102E70005C87C803DC1A10D36DE2983A81F3EE68E0
:102E8000F82D093962D610779AC5FD9FAE59E8DE54
:102E9000E42DFFF2C896FF31BE9877D78D3716E93B
:102EA000FE2DB3160B89972A49F998F97BEB4C80D4
:102EB00009CCF7F5FF2110C0B30F818C8809DF30F2
:102EC00041EE98224282BFCCB0EE10E0FEF3FAF958
:102ED000306032B30D7657B9A4A2985CF9DE89212F
:102EE0000486F4663A66A04904FD5F2826676846B2
:102EF000A1D3DE9818426260B7D689EE2420EC1B7D
:102F0000B3730488D019BE59DF28CD8D5A56ACBB97
:102F1000409CEDC804427EF9DB80305F01D8A410EC
:102F2000BB58FBBEE8D3F30772B0C231F61060E0C5
:102F3000511EDDCBE928232D91BAB08F86F7487852
:102F4000100EDB8040703093D311D310BFF16D4968
:102F500007D7462DA0D001B0390A82275612443433
:102F60000A66961966D5216640D3ED28F9300B9391
:102F700009FAC6B40EA29219B03AE4CC131F118C10
:102F800080453F6F46C02258045AA2C20880C03113
:102F90008A66A919405C02FE489808030481801FD4
:102FA000403002316E447B0912019E712202B2FA56
:102FB000BD988829DF588185100FBBE8D798F1F8B4
:102FC00098302564E69BF536EFB20C9007F0017956
:102FD0009865A8DEA569E798F34D3C10BF208F30B7
:102FE000413A825EA5329308B650DD66925DEBF3FE
:102FF000DBE0D4328FADF3E52B8F301B46D341CFCE
:10300000B34CFF11FD4CAFE71798B98E964091B0C5
:10301000CEFD7F80733026C176C9E3D6EDB521E7BA
:103020003013010270B3AEA4767DA48006B9C81334
:103030002210E23280206E881AFEA82124BE65CDBF
:10304000F6E58085B9EAC85EBD91633AD65D03EFC7
:103050009812430360C6810CFA11350220FB5AAD69
:10306000109187DB16F3DBEF713019ADA666DC300B
:103070004519B629BA46AF803B8B209BD1FDC9AA22
:10308000CD71040EC0FB3947DCA8A708E02B37F749
:1030900032C071300099C90310D3E0B409E8740557
:1030A0008369A26EE3FCB6F80D40CFB20B08140D95
:1030B00030B6342F42DDA80825FD500D9BF932A013
:1030C000A0EFA10610DA1CF59811FE9894588AF327
:1030D00027E6FA70F85C3009C4E153DD148CB8DBE4
:1030E0002674822AF860808884410DB737226AF8F6
:1030F000AF11F499400448328460B4833C069F5C6D
:103100008D041060244F3D020108FD7F003072469F
:10311000704B53BD4CDD0104EA98E0312C0E513068
:1031200090E03B017120034E7A30401EC083F58B46
:10313000647B9858FC7F1C30D7AE83AF17BB836D80
:103140001F3D98848081C4CFFFFBB6239B301804B9
:10315000F8239BB9D8FBB3C844776BB12340B5AE15
:10316000C02587DC8880D3858411D8300481B6DC03
:103170005C7F6B3701437839B301EE226282FE0136
:1031800011F0EE851716AF08E12F0B6CE72122A096
:10319000A0108011FE7D3040288834099C6CD70532
:1031A000362BF788D4986860A210AA723240626801
:1031B000024D788610A71A30652EE253E3CACBF58C
:1031C00034F7FEB53A37D3E1925C4AA9026DC608DE
:1031D000FBBC6DBB44109A0A9A386D3B201E7B8164
:1031E000316EB26FEA983CF9107A5D2408BCD48342
:1031F0009BC60222BCB5BF52FB3BC490A0FC68B486
:1032000042B95D3426209B1AE2EFF5C7B09C66CE2A
:10321000A8013316028844D3BE9EFCE7C85848F381
:103220001184E6800905F6F9BC98B830BFD908E4E6
:1032300002148C9ACAF4068D738C60014CDD30DA6E
:103240001202F1D9AA210CE38A86F4B714B5AF01B2
:103250001CA45C13120287E6F960F8BD98A04AE14D
:103260001ED876580F680DFD9810E60FE2402C0727
:10327000F1BC43B603DF733DA007D2F0408C1A5077
:10328000D30C9D23F31EC466C80FEF6F6B28F9EBB8
:1032900017407F0FC9D5B66DAECF013188D75B140B
:1032A000D8027166E0BFC1EFD312895FA8D33ABBE1
:1032B00082413BCC8FCAFA80E973260A21EE3BEAB1
:1032C000EFDECD31B0AE9615DBD7FB9B1246B48056
:1032D000CB4E8EB3FA38F74B42440C5AE2E2220846
:1032E000FC31B3FF7D31AF02E538827BC975EE3426
:1032F000FF20E7D0F985DA246719F3DF325DDF7943
:10330000E0E71780D364B0C6C0FF1858FFB620E3CB
:103310001E116CE4C9F86C66CE31D1C6D3BAFDCFAC
:10332000F8FA0C7FE5BABEC1BFDE5AB2807BDB1271
:103330007F5CB1A065ACCE4025590B806DF2D0FC0E
:10334000B131984409A1F39EC279E0A0D32686E06A
:103350004B17C9FC640206610FDFCCF632DCD46681
:10336000FC321BE896190C47DACE19948BBE103943
:10337000274223C1323E248FF3EA5158F6F8D7EEA4
:10338000ED0837DE316BE7FF1470F86CD162ABCC1F
:103390008034F0C57AEEF5BB9095E6E579229E9BE8
:1033A000DE408051771BFB661960E3A54670B8F9D3
:1033B000DC9B82E5A3BD1F1632AE56DE4DAE5937FB
:1033C000AC81CB341866CCF36860F192706A736E8E
:1033D000D3A308F553DE5CEB0670F9CC3C9365CDC6
:1033E0005096530125EB5A885F3C777BDD7A02C605
:1033F0000880ED2028FACF98107BE09C3FBC44D594
:10340000C47F71405E7B88815DE596D7FE1642FFE2
:10341000B69362F8B3A8B508577309FCA7850420D2
:103420001453D45072ED4859A1C3B3CD05C69601CB
:10343000E3C250586E420B43BD95B4517F39032609
:10344000800D18E8FCDB2002FDA82E65242E819853
:1034500037C918FE4101800ACE7FB3B0060CB68191
:103460007211FF2A03150A08C14161CB04E037F34A
:103470008901C78220EC0A78F957BB21201015E496
:10348000B88496C7E59BE365284828D3BAB1CCF544
:103490006101FD1CA304FAFEE8C47B16818B400881
:1034A000AD029403E0FC64789008051B88FCCE9282
:1034B00033FBFB654462BECD2CB04FBECD4008301F
:1034C000FFFCB3A9BAD43343CB19DBDF3FA9D30642
:1034D00088B1FB25E0028B6FE0800277E8B811F736
:1034E000C8FCE62826DD3FD978FA2228BBCE16454F
:1034F000EECBF10265D880A12C10F2E866FF5BA646
:1035000081FC50FC8CF26440C5F9CC08623C9ED82A
:1035100090FABFDBF0EDFF9CA76FB496F50D94C752
:10352000DEA8FBE164991C7E9463DC64B410E8AE11
:1035300028D49D00E0FE0894E363DC7D63B9E8B322
:10354000FEC504409E7562ABC00435CF602CB3331A
:1035500059FF01FB2D77EC24FC5092FD8CB3C2B2D5
:10356000A559B2F99FFA63EBFF0C5E5A3A48FEE2A6
:1035700030C96D7F08FB3E37C10DFF98BDFD9E0130
:1035800065F96E8F7E7F01C55BB330FD1FF1F2BC24
:10359000B540FBBB1ECE7870FCC39529409A8BD9F1
:1035A00018FBAB4708353B1067E62601C8EB123520
:1035B000DA98B1FB7288D02EAC2A2E58D982FD7EC3
:1035C000EBB342397F0A616309F8FB71B48AF68C68
:1035D00080C2DEE85E5CFBCCC7B83CC5370D02B2EA
:1035E00008B6D4DF6096327429DB36052027EB9AC3
:1035F000802B56E5409E0410B5E6CE2610F8F5DD8A
:103600000218E54224B24040E03532AB9678FC6FB8
:103610006C1D60EEB33C169D022FDAD98158DBFB9E
:103620009FD64E58A3B7B4E890802E0C090972A11A
:10363000246DBF64B6A578FF7E9B2DEC71822AD5E0
:10364000692066681075E47CB7B948491170B60204
:10365000AB3084E82EF92030FFDBFF502ED5056615
:10366000FB1860E403063015D7ECD59FF88DA01544
:1036700001329F049C50133C026C79BB10D435B3CB
:10368000F8040A234028FA05A0EB17DE59C1494186
:1036900011E2D54F3D04023810021CFDB02801098B
:1036A0008406C05ADB7E126061FD617F0482413274
:1036B000688092DF1208FC7D72244A824CE810F385
:1036C00064D1B390B32D0882853E932FA520331685
:1036D000FC6788922E74DD4410B76BF96304F66AB8
:1036E000D39D21FDC0FFA9D9BFA4A508F3D30344EE
:1036F000F8044168B82D5992664010BE838DB0B26F
:103700002F232BF51511CB7D9037F6846014F673BB
:103710000CCA1EB3654CFA02CA0069FED8DC01D996
:10372000BEF93A21203636CEF9F62F1BF90467F997
:10373000AF9FCA402022C8FCFB1B63EC14DE1AB109
:10374000F8DCEBC4FA14BA96CFDBF83C88D9E288EF
:10375000D8FE0CAEC07BB1039511022CE410F6A389
:10376000A0F9CD598F01E6403F9683ED7AC8FC91D0
:10377000EBB5046FD9D420C6587E6F0F4037921630
:10378000911F8B6FFF53DE14DDA00892A9B120F6C4
:103790005790F9C73433BAF2CCFDF906AA3902DDE5
:1037A0008A106E0FD960F9F9F9B308972C0819C47B
:1037B0006A3F0837BD3DCB13214CE24068B0B3D817
:1037C000FFBAA5CB048BFD226250DB38097EE88C62
:1037D0005BFDDA9103B4F8F0FEAD626D88010D2C4B
:1037E000E612FFFA3226C020D4E21F778325248810
:1037F0006B81080ABB11B00324FD304258FD8B07D2
:103800003BB10C6565C099F65C47EB9C78F6CC3C07
:1038100024CEA178FC93B310F9AD20A510371CFC81
:10382000CDAD688B56A0DD201EDF4C0B80413CD710
:103830000820AC98345FF6E1A0204F292FFE42B853
:1038400010B38BF3AB6969051944AD04577CC06CA8
:1038500017B049B85032D50466D83DC9F6150416DC
:1038600069C8995C0C1E88B7C226349014F3C9113C
:103870000A5CF9D268FE1910C44BB34C8547F3FFBC
:10388000601E80C00730D70608EBF90F468BF39215
:103890000512DFECD00920B91AFAFDE62089A866E6
:1038A0000CE6C408E8B674BD18080F820C80663CAC
:1038B000666EFF0A50E690192B0112FB3296B3B0E8
:1038C000734CA001FDB1104608041ADEDBE90C823E
:1038D00005D9487FB35E240419B0EC4050FCA6D44F
:1038E0000901DF25D71ADA8467BE9D0424C0801041
:1038F00033BD9822B841E2BD9802ED5101093D98CF
:103900005CB1F97EB1D21D23C61D3D3A406FBEFCAD
:103910008088F8CB35CCEDDF1EFFCC5F326766C503
:1039200064ED5DB9C4EA98583DE00720ED16C00388
:103930007D987965AD1948979210186797FA7F08B6
:10394000014208253371A067F588081009E098A1A5
:1039500080D93A6BB38C56F81804D7F6321168B494
:10396000AF80C9B84269B3BF60EFCDFF328002605B
:1039700019FE980196B3B50F589106BFB798011C70
:103980007E4906851926E8B2901F12400278107F02
:10399000B69868FD25FCCC1810B1663E956466E9C2
:1039A0006BC0E04166592666BE98D869FD97ED4B1D
:1039B00098BC98CE2066691E44C1089BEEEFF44C7B
:1039C00001FBCCB880FF7B98300510FB25D521B7D3
:1039D0000D3BF6D6982025CFFD30C210C0D7084148
:1039E000FA618489013FE0C0983FC1986C42D84099
:1039F00066C7F573026419A699ECD9A0FF0AF418FA
:103A000032B3BD98E42C46439EFD3C8005F2EF4D59
:103A10009870E008B7AF9802F4980CECECFE044BF9
:103A2000F7CC2071547DF988AB6888CB7CDD986831
:103A3000820CBFAB9811CE986DB928FACBB3965DC6
:103A40002CC7B38B667C3BCF98D683260166761154
:103A5000D304E5B301AFAE9812F6982140C9FACC71
:103A6000E35D52A6E250F698E081C4772F3CFAA0BD
:103A700007F08006FDEC2011D316FE987F26300C4F
:103A800052FCCAE0060DBC9888667BC4BECC7DEDB6
:103A900006C14018C7D32C6608BF5998F862B33CDA
:103AA000D5B305778D98B3B288FBE50106EBC0046A
:103AB0009AFACC228C0ABCCAF69810C0C9FB327E96
:103AC0001BB4DC09FC98B2C8CFE63030C2034E13F9
:103AD0003026AE94B480F59869FE9807F0FA610F2D
:103AE00018309190FBC634B60665462CBB15B1F96B
:103AF0002F2D4BAF1CD832608E77C8013C667B1CE3
:103B000084B864CDDB38F8A1DE98057A9881BB03D0
:103B1000FF624AB35015678DF60823CE3009400482
:103B2000B83094198463DF1140EA9801F2986C88E8
:103B300012FE4B9B309804FD9831D9B008DE9AAF45
:103B4000459BDABF58FE326DBD28B9CA047F3630B6
:103B500070FB25C8301E2FF298312C0419A05BB2DF
:103B6000F3C840AD071B6BBD91BD98085C3072492E
:103B7000FBC4F930086BCB302010E330BECCFF2201
:103B800098875F66A1D5FEE498FFD811FE9FEF7F6E
:103B900001E530849F9EAE8011303786C008831BBC
:103BA00000AF6816A40EBC302BB3CB98ACBD9EED15
:103BB000B12808FD98012BDB2BC82CF5E71804264B
:103BC000C0F4201822826AE481801092402D9079FE
:103BD00030A45E65BCE0B3C43E4B4B66651D3FFF41
:103BE000A4B18B76C54BE64B4BB36020B6023F19B0
:103BF0008CCA4752AF409B4D7064167F46400F4FB2
:103C0000348007A020D714C0FACC0BE041E562F85D
:103C100093CD7D0401BEDD49E498E6B30ABBE90813
:103C20008182109102E7526C4C79A9149106A1AFE0
:103C30008A0D9844D2241019FCC976B3142C08A616
:103C40001AA0666C22FD81E504EE164010F59882FC
:103C50007E05280616A4DBE9327758B2FAF830D58B
:103C6000F6169608E72990C8261C26B14DE07E1866
:103C7000C9D324F3BFB0C198EE0960FDC9F992D64B
:103C8000A340737366FC98C4797D20DA0641F23054
:103C9000089B6606A26E263084D8FFCA3789D2FCFC
:103CA000E3588CF3FDF149A00131BC02C00418E9CE
:103CB000666824E010365C80BE9829F3F1FE5EC48D
:103CC0006FF6894F1330DDA051B384DD670432C233
:103CD0007D30AFB79850846DB2B64DC8B9FC95E64B
:103CE000987E4B41941CE12D8D65A9D010193C673D
:103CF000E5C8756436F388807FFCCCC001398080CC
:103D000018FF4D9803F3290BA6F3FC982AFE9F6930
:103D1000FC42C8625C30792C9FB591B83610F1C076
:103D20005FE498F3E0101140BF9D301244242BD182
:103D3000BAD6E5B0F9C86FC9CA05F3AC2196C8D3A5
:103D40007306058130BCC49CE0C1012C706666BE60
:103D5000985AAF13AAF84B19103BD4981EF3766CFF
:103D6000C82C43CB989230F0269D90100F62DC3027
:103D70001DAFB998E0413CE25DFEB330FDE5186B44
:103D8000F27F9ACE566681AFE9C1E630200C6BF324
:103D900028EDCCF2C876E689FFFEB27F9A7891B31F
:103DA000BA1119C69DEC9805B0F371C008191968CD
:103DB000C9020CF3E18C06DBD398906CD0AFFC8E7B
:103DC000C7D7E0182CBFD53777828DDD2F048A79CD
:103DD0009865C8DE98D7B001A598D019DE98197AF1
:103DE0009821CAC82E1640678BC01914F380619DB4
:103DF000E049D8C0FC6EECC098FE64FDCC7D697DC6
:103E0000FAEB1978FAB1C439303C72C41CFF199826
:103E1000B328FDB7C0F0988616F996AC09AAD5224A
:103E200023B819C8AFE31B1065B320908F76724397
:103E3000B2C8FFCB5F9166FD980A5E983410C0B39C
:103E40006DECB220246A80DBD0FEACBCB84166D8F1
:103E5000B210873830410401799810E0CC020CCFC1
:103E60002819C6A36BE99805F6AE68B664F4B25893
:103E70000E03E4016B9007ABD13AE82001F3AB11DC
:103E8000F298F162906FEF98073040165E9876FADC
:103E9000491C1040EBFE6281D6228201DC66E30EF3
:103EA0003FCFE5FEB98440BA44FF516B28EFBF8D88
:103EB00098D470DF7F05AB89248CBC80B3B8307296
:103EC000F3080CE159C6FC30D7B120E70C5AFD6865
:103ED0000A77163090EBFBA73C8190B010B228B364
:103EE0002E846DE098A921E289034404B320FDE902
:103EF0008280C0FE0D3022874150B984B01237B5A0
:103F000009F3FD21D864E52E9EC76282E946C57893
:103F100030055093A8FC1814023D72161C84F3D788
:103F2000B18E1E5C303D53AF169752E0F230F05721
:103F3000649D98F09C0DD1FA97B6BCA8299A0FD928
:103F4000C7FCBC05F1DFEF5CFD8EA0DB55426B29A1
:103F5000BCAB4CA1D8022C0144A519DB6295AEAFD5
:103F6000128C88BD8D46A20189FD7208DC30B60234
:103F70003699E6CAB00874B60419E0B411E1CA690A
:103F800010126693E61139E8B2F8F3C8E0AF812F5A
:103F900098D2E908F30BEE5A30049A66A0AB68D7C2
:103FA0000C96985DC8E86B64142419EB400E48C069
:103FB000982E76302058F85E9A15F9E5693517384D
:103FC00045D16AB3B55050B388B60BC4F930104729
:103FD000D30D66F384A0E3D8E6D19AB358EF52E24A
:103FE000087C10D4B35B257B9832213AC01098F737
:103FF0004B0444A1D31112B388188E01FEF71A3076
:104000001278FDCC841EE1667EC410D38C51EE6B19
:104010005DB8FFD49280E25EEA5BF06718F38AA293
:1040200080C833B58BD32CC8121DFF98FF2485465A
:10403000663839C4FAF9609066D7D8FB9A451AA059
:10404000FDEC8BFDA1E7669EFA7346F37F2CACF97D
:1040500083EBCC51B3B13CD1DC241312621739F895
:104060003047FACCFA7F331AD28008DDF0612C4455
:104070001888FE42F365379BFA40580FBCE5CAFE2C
:10408000C598FDC2C3C77FD86A108BE2A8FF62063D
:104090001C3AAFB78033F9FC4BC64B192C904CEA55
:1040A000C933F43DBEB0B2FE508D40194B3B048C79
:1040B000294FF6DD81BEB76767FAB8FB66832063D8
:1040C000FFC9662E620250CE0AF88F7F28B2FD9B90
:1040D000BF040163A9F52A80678AA5704B4C41B0E3
:1040E00056E610205CF3CA0610F69ADCFDC84D3384
:1040F000F000082FDBC0158792B6B823DEFD051847
:10410000143C940A482FD82C52CCA816B450391914
:104110000C0B300CDF1838A615FDB1B7032743612F
:10412000811501B30698670130CB4F495AF451BF4E
:10413000D5180442C00FD4DD8250FB320813F3E9D6
:104140003FEC035FCBA04F53FDEC406AC5FECA6C49
:10415000B604029D94528FED671F66D2B79ACC5772
:104160007F81DFCCEB4BFA1FF3621F37EC6CFF183B
:10417000FF5F55B801F69225A6FD9D175A3867F3E3
:10418000AB48F9616F572998F7BA5AD05819D758E0
:10419000B0B7D87DA776E388FE3FC6A43EFF63FC98
:1041A0007D2C8059CE48672D9A408DF87A17C2DE53
:1041B0003C79E12233C2F562020234CF0027D756A0
:1041C000AF102C4BB802F9CFFE7A68F9C5D671044E
:1041D000C6CF13FF5D30FA6176CA0EA031494FD8C1
:1041E000F7405DEB988810F3217CEC4CC0FE7C42DC
:1041F000C7FCCBDD591861C69815DE98AFFFDE927B
:104200002F1DE47D63623DB1D878FD2518667219D3
:10421000B301BF74D8B2FEBAF0CF302B8FCDD3DB51
:10422000D3D8FD1258940ABEDBF5F13C89731330E4
:10423000FB615FACEC806DE238B1FF75332289AE73
:10424000B3010664C51B8808FC303BC2AFB387D2FC
:10425000CFC819C2D5FF808D69AF857BA5B540F366
:1042600021146C3888FCD3403CC4C29D76DCE8F94C
:1042700002864372C520E588118CFAE520CBED1942
:1042800004FF51A3FBCD66484004CD6C8810084F55
:10429000C25CA2E55C8682DC9D41B41081ABA7F8CC
:1042A000FA7FA88210E49BFB0182C95A5360FE503A
:1042B000011A08800C20C43F9B20A414391081BD32
:1042C000A8E6290560F6146BB058C11BD244E42857
:1042D00076663001CD1E0C60E338E61043EE6A418D
:1042E000625ED59808B784DE02A80450D3F99D8C8D
:1042F000A0EEF00242200D43FB21700A38F93FEC9A
:10430000107F8C6FF2A13F74EBEC56FC4060C0A3B1
:1043100026E6FE7FE3FA13F5E02091A25D6F94415B
:1043200081F2CE8040ABC0FF0311F6991020C63D4C
:10433000F24047C6EDE59FC07E3634FE49509A1DD7
:1043400008B1CC9325CD5C4DB95BCEE0F81B31D1E3
:104350005FD8B540A776A450FA578BBEBE0EDBFFE0
:10436000B0FD73BF0A7B5B021D67C004206E612F26
:1043700050FE53E0F9C37E59CC20ED8D90FD8AF2BA
:104380005520C7D7B02099F34AD718FB3217EB3224
:104390000BBFBC14B1FB7E5849019ACF41EFB1CDA0
:1043A0005E5862E8A79FE5E61CA6301477A9A8FE30
:1043B000609FB64916B67D020457DBAF6EA2240794
:1043C000B8FF20BF48E98D8F48B40C4A1DD0D4E314
:1043D000FD144E6989FD101298F713017421BA6E0D
:1043E000D7F181280906B648F88A49405B97602CC6
:1043F00095205FED81FB22036EEEB4203B52DADCA8
:1044000098FBFB60F88FDFF55F01CB9DC015F5973A
:10441000C0CAB3A037F85B19C06FA80130CD10E84F
:104420006604C753F23D44D003E1F459626D65A0C0
:10443000012DD4481B884C08CDD11FAC28902920D1
:1044400002F0C0FF8005D3A028189611C09E54BB6F
:104450004656D60B31BD96C460FF9B666B81408883
:10446000818921DE08FCE587F01E3BFB7810DA9598
:1044700007F16CA383784CB771D30180AF902319F7
:1044800090CDC63F8C0FE0E0013C6F58FCF9ACE3E7
:104490008418DBF77F0636D6036031ABFC8445F920
:1044A0000C9BF165FE0840FCC089DDB38468B3E86D
:1044B000800401B3CFD7A5040815682E1DFE940211
:1044C0004CF619C022D1A682C00930EF70FD2056EB
:1044D000BD4460F40A490DDBB8AE203463F0C18DF1
:1044E000FF7B307FFDD315CD9809FE9835AF23D6DD
:1044F0005A9C899918F312A9FF2920092601A4FBC7
:10450000806FD3A5B90C6DA4CCD50D95CB670C9F4E
:10451000E967D5FF868164AFEC043C58F4664988AE
:1045200080A0BBB141798675FD1E53E52883FE8DC1
:1045300019D7B111FBAC0777EE5DEFC45C54A4A6AC
:1045400046829EE544D3F3F10A620120F2E1FC1AAF
:10455000D8716E0F0CD33DFE096CFE0A8F5A496963
:104560007B0B77B7AFEF3498FDCC8B7DE6A7A64BDE
:1045700002EF037CCF8D8029B03FEAF884310DFE35
:10458000980B0B61355C889DAC2604CCC60284DA9E
:10459000A931AFB3517BFA8E477CCFFF706842FBE5
:1045A0002A062C02F56604FAED814889F6200132CC
:1045B000F9DE98E6C40378BDE09C1C077040A0A318
:1045C000F368F3CACFE14A84F4B70DF5980379A5EF
:1045D000A7AD98201FF3E4013C08386FE798F9F283
:1045E000CDF30640C766198B88B30810341B719F42
:1045F000BFCD7FC68012D3F38424300F21FE8011FB
:1046000005B2B341D1B3C0BB82D64B1152B308FF40
:10461000DA8C197961AFED3F2E3ECC94E5230CFC8A
:1046200080813005B8FE06AF9108104A81AF01AF16
:10463000F43F98F7E78179989466FD0E231966A5F3
:1046400001728C94268240971529FECCD0D3FE6E41
:104650004D2009366DCBF9C5D0BA95B7C599B86963
:10466000195CB3ED77914017570479A5A166A8CFDF
:104670009D3219F0FFAE8ABF232FDB23E023FCE03D
:104680008D60FBAE587BC74D778C1BFD5DFEA0F6A1
:10469000ECFB497FCD05DF62DC636819050F90C331
:1046A000444D2846B8ABF304735657AA416F51DA0C
:1046B000FF847FCC88209B11E10C75B2223472807C
:1046C00029A1B5F9405398AD23EE9E8811F97F8753
:1046D00029F3AD80B7115C6620B3CAE70B39EB480C
:1046E000BD98099D20778C10E2C6AA890A1989F61F
:1046F0003001C0FB9ED2FA401EC48378E56A419324
:10470000C230F3DFEFCCFFE007090FAFE28B7FB0E1
:10471000121ECFF198C65E98111B19F8989646D6CE
:10472000DC302C73EF21E570AB77EF7F42F95AD381
:104730006FAAFC80EF2A888130EC1050FD97B324DB
:104740002C826EB37FDB75F22E05F1C1A0A6860622
:10475000128075D31013DB640865190B74A19CD308
:1047600019E8FDEE8A2411E730408808E92141224A
:10477000E520D29240C16902F38B74B32104BBC619
:10478000ABE077D717E2C918DB13FE8248FE2E2371
:104790007A300212A4F916E2F4BBF610B5AD33DD9F
:1047A00075150873227760DEBB09F2723901DCE00F
:1047B000D38897870EE8F9B885FE03308203400C52
:1047C0000A410AEB35FC988C8CBD9E988377A9FB37
:1047D0005EE7F5CB1CC0E053895CE14F0A609E8F19
:1047E00081FC205CD4E8A602ED0448F2B8395B17DE
:1047F0004C6E84682DEB5D77A62FE8DE2E1A408C78
:10480000CF8D27DF6A0D90293F71C2FC8011A0AEC9
:1048100008431D18F84360114084A6DC063524DEE9
:104820002BF644408805E7666BCA5967F42BCF1115
:10483000507429CAB4649614FCDF7FA680B08489C2
:104840007EDA12F8E0013DEF4AD21E46F59860D9B3
:10485000C8BB718D503C8BD9FF8A4F36448DA20D59
:1048600080E5D394A7C8D305AF9B5EFA98103DF8B6
:104870007E2C08D3D5E561EA38812ED636FAF08B46
:10488000ACACA54A60801EA0ED6FD6479E6B69CD8B
:104890003049FD2EB30200B370C0842C2805B3B894
:1048A0005DBD9880DB8C82FA4B02D3FE9528018A8D
:1048B000118F45FEB96284C84FB30AA08C80058170
:1048C000323097FF11EB558048C008681DDF5C113E
:1048D000D9E8EB100814CD984666B352ECFCB5034A
:1048E000A8238021AFEDF4CC9A0813CC6D97C8EDC6
:1048F000D3D9C8DE10FB8C28EFF040F3B6846D2EC0
:1049000081207CBEF3B3FCDA76BFA8BBFDEBB3031A
:10491000381487D6C220E8BFFBB2873023BC983D4D
:104920000A11AE9BDC14B4603DBE6670768080FBDD
:104930004913AA33C5C6B35B80DDB3801DAF1659DA
:1049400079C8C8FF24CF6D9F9504818408771E30F5
:10495000491A4C2B656608EF805F038D8359C87731
:10496000B6985844E5B396C8A83CB21F78F98409B4
:10497000B0BF10FF322304024C829B91E9169FE0E6
:104980000B04242084B511F665B001EDFD594B43AD
:104990008A4802C469FBDB0508AD662835AF88FF8D
:1049A000892008A0FBE0413C7FA798C4A7100B7F9B
:1049B000B498F120A36BE69880299C5EF7420F8A99
:1049C00004E4C845C630A4E7C677AF6B01F198F49C
:1049D000AFFC35E5E77D62200CC788016BC57DC75C
:1049E0005079E5E77E7596DFC1B40AD337CD07CDA0
:1049F000197ECCE6B950FBDDB30B81404C5D847869
:104A0000B30F2360088C779E4B19C64022BB01561A
:104A1000802A86C9E6B4FB493FE22084293004C0DD
:104A2000B0FD8688D33E5910490C01F6E81228578C
:104A3000C136C94924C2CCB353FC9B626AD6BBA021
:104A4000506594DC9D13516D99C812BEFE4130092A
:104A50000602BCFADF6D66FADE8F8537D6E323C720
:104A6000F83B372AB6FF2EED32307AB1FD91F6824F
:104A70003770FC7192DE98BB8037C8602EE5C0E5C8
:104A80009F181BA27E7F50F7A02733AABCFFF79B7D
:104A90000588038D328983EF0CE6600130B9FA4254
:104AA0002C6A81F420442D24E57AE309B53590B5CC
:104AB00010F51668FCD5E50F733066A7343E5840F4
:104AC000E8B72CEAFB7F592890292002BBFE5CF74F
:104AD00077213098770B6014E6C8468B7086CAFC45
:104AE00082B606D01FF7FA55277AAFBF2E9B143037
:104AF000A4CD6A4A95C073D3E0AF88818921D7518C
:104B0000FC9DDFE6986E41C8D7792019237FCCF24F
:104B10000502300BD3F65B1ED05BB664C806FC30D2
:104B2000359EFAC077DBE5C8FA155D0768F3B581F5
:104B3000D212E30080B35B3028A818FCDF2DC83EFA
:104B400072E6C6A9F9DFCE98E3304CD77B0464DE69
:104B500062D306DBE3413A5DF8C1132E6BE0140823
:104B600029C8EA8C6F92C8E6B7B685F5B00898F800
:104B7000CD4A20C0FE9885092D2BF38E50F88893DE
:104B800061C82069C66FDAC4F443DD5367B37E574A
:104B9000C817AD9B6B64C807E6C8360DB893E2989A
:104BA000ABF0C996C1BB692CA0B7B3475F13EDFF4B
:104BB00080810E19F36B2CFFB2C8741FF8FFB94542
:104BC0007BE7981CED9B0E011252F370F641D5B8AD
:104BD000127FFD4621551B771F0694C8E4B220F3CF
:104BE000540AA768E638FE282FC2F1C4B83B2980D2
:104BF00022B8E252EFF368B4DCDBB7B16AF31D0907
:104C000055F717E7A101A14F1A650B207F11EBC6DD
:104C1000A3DD2D809929FBEA46FF11B01006C84894
:104C20001801EF236080F7A516C8029019F30E60F3
:104C300082118F6834667219D50B7FA1D73BC810DB
:104C40006052BAD282DBF6F3C808BBF038C88007DE
:104C500036009E987F93B8F3C883AF1833983FCC43
:104C600013ED1D0B0778305283D303F647F080C84D
:104C7000F69860FEBC985BE37A9884FF50E540F3B9
:104C80000764C87652B3035B24FD90EBD3025EBF8A
:104C900017DF8B88413010895C306EB3DC42888925
:104CA000F727C208183B898C82056E35BADDDE0A0B
:104CB000A10BCF6E936084206DC5CAC548BCF609B0
:104CC00030D74BFA9DEC9804803810096FCED54050
:104CD00094EE6BB76101CC8BB71920010B96EFBF37
:104CE0009E3A5EFDC62221BB0437B224F2302980F1
:104CF000A5D7301BAA7D6EB1C5E576A7151AC8AE3B
:104D0000638473B0154AFFF9306CD9667203048767
:104D10005183F8606B95C8C722128EE8815DFAE076
:104D200098016CCFBD32910AFDC55BAB08803CC7D2
:104D3000EF84326DD564C24DE3E0ECD5F9E698DC42
:104D4000E5CA0A2DF32F52BB12C29836E17EDB7BF7
:104D5000B386CDED6CEF88155658EE98844C082339
:104D60008966D30B3CB20D8409F6E5B0F880B9C86A
:104D7000E9010B6157453AFCC64057C50BB4988012
:104D8000310C6A6677BF538D1BAE08101869CF715E
:104D9000886044802D25BE1239C73EF3304260FD45
:104DA000DF3DC8037810B78B98A3BD98E847D49F20
:104DB0004A9587B01CFA0AE841DB74B2C856D3D9C9
:104DC000B37E989D81B978FFDE98667130F9C8018D
:104DD000798BBF087D28AFD881108CDC254FD38319
:104DE00060200C69E0CC1A659BDE9EB2D8F9304C8D
:104DF0002BF37A49C40257C808590002666B03FFB7
:104E00006284DE4910B3FC052360020C81A2E3C674
:104E10002FE678334C8105310BCC98F3FF7DB255EA
:104E2000747EE7B3EE40FF018DBBFF2CFE20F6E75A
:104E3000FF16783640F324F36EB5B92270C69BEFA7
:104E4000B32828D3CE03C64880FCC205FF50F92EF4
:104E5000F6C46F6ADF38D8D8D8FAE193EBFF28DFC1
:104E6000B344E758FD20636DD373FDFFE66675DE3E
:104E7000FBD4651F66EE92CEEFFACFFBCC7E3FFAF5
:104E8000FB29F1FB71F3A0662CA801D79B062E58D5
:104E9000B70F37C23F66F66408ACA7FA04BCEB73E1
:104EA000F3EB75BE02E6B1671DFF96D1E6D349E785
:104EB000BBC6A1FB637FF967182BE3D398FF771B71
:104EC0001299D446112EFF6ED16E607E966DAC6243
:104ED000FD58CD58A7EAFF01CF6CEEA8FE61C9A02E
:104EE0006CF7B310C86DFFCE4EE30260E8FDCD3322
:104EF000E8CD85CFB6592B80DEEEB2405BC2F8FC20
:104F0000153B1D6CD953CDAAFF0A806AB26E86B3D9
:104F10001816B304E68A6798EA92A712CA3F9D85DD
:104F20005D65FEC7BF046D64CF685AE004991CEA52
:104F3000A60106C5F3F765B40169F736BF30FBAAD1
:104F4000580852C640A204B67BD7E8FD9CC4966EB2
:104F50000459556A7A10ED2DA21B81B3F983BE2442
:104F60009508BB0DD38264BDA49415E893AF0231BC
:104F7000781766800383EF010494EB06DC8C200233
:104F800090082378014A70697488FDAFF80442C123
:104F9000206811A1A64CB421858ADFEC622801B3F8
:104FA00089C765ECA2843D9D984441333681409188
:104FB000060C0771AD27D528A438FC80129E5941F4
:104FC0004008803B73391F6EFF10903FFAECEAAF48
:104FD000E96490FEC2204706ABE201EFB4FDF85051
:104FE000DFBA1C8EF7C4BDE501DA40040AF7E0EB36
:104FF0006427DB8FD5FA161670E3122FFF025CC40C
:1050000014F5D9C8F8FEBB476F18B55EFF381F7896
:10501000FDACD168466A45B020BDB1C065F6FE184A
:10502000FF8EA2C61BD1800255980189771020FE01
:10503000631F4D63AB7808105895FE9F1863EF2DE2
:105040001B028CCEC6C3B8FDCAF3D81B597E0C8B8D
:10505000A90110FE07A8F8C93C5A88CFF5D6088CDC
:10506000195CAD63B8FA93F2DBC9C305FFA0908B5E
:10507000657E7F02E37C0ABFBE087A5E10D956487F
:105080000358FA67983049FB210811DACDE3CACCFE
:10509000A89DB78159D32046BA724B80C456924519
:1050A0002DE698E6D2143B510888FF3FEC5F7FCC99
:1050B0004A5B8CEDBD5862205ABB67EF31A8F9619D
:1050C0007ACB80CF2E820120035F70D8A0FB5EB325
:1050D000631EC0D888FEE17A84FBD6A6C0D350FFF9
:1050E000E3CD11DDC21088F9B88F7B6DDCFA63ABBC
:1050F0003980556B60843FBBB27096B34013F76341
:105100001004B112165848FDF2A8CB81B274D74FE3
:105110008B1B69EE801DF3F53FD992B8FFBF6799ED
:105120004EE413E76799DDF9F85BF0B5FCDD064066
:1051300005DBB6043F9C40F635377E5BADA09C6B2B
:10514000D3671065A1A2B39FCB83C2DF333A38B2D5
:105150009DCE375B51F840D2D97B8A1296D94099BF
:10516000C28EF864E411B1567FABF8122C2E5B931B
:105170002840C7019322E3FB0880103540B3820822
:10518000A0CC34FBA205580325B321C50AB23D6368
:105190000B00CBD580D52BA553EFA2130260115085
:1051A000401AC1292CF90CA00132C0D91E1064C6C6
:1051B00020F35CC8FD3921AB074010E1080470B949
:1051C0009F223AA901384E0145CE1740CFE908C8C1
:1051D00077BDED4C092A0329A541478C89815844A4
:1051E0002A28FB814A20D8F851474E6FF2A29AD460
:1051F000F7CCEBBB7FB2BAFDCA0464FFDFB0FF2D72
:105200001978FF008F3CE3CD8DA1FF8F02625E9C79
:1052100041E42981F782B580398CFB78D9FF10C72A
:1052200080FD24BB8540116BA67A3DD4E27AD8A4D8
:10523000FFC1E1859D184D8190FF906FB840A0CED1
:10524000E55510849A459828CC0216384F6C1718EB
:10525000CE0A7BC2FDEC3310FDCD5CE820F7666919
:1052600014BF76E802803BAB8F9818DB490A0967C8
:105270003C0C7AD4FB5989BD7AB504001CC6BF45E5
:1052800008627F68B2FBCB198DA9CBF2AC386336CC
:105290008602243FECC8FE806B2C44FFDB2F019874
:1052A00026814565C89C026AA4099FE2AAB7C5F396
:1052B000300249DB01A3D9B0F9C7B48B4DE43C3CC3
:1052C000C7FC93D7D64B20EBB540217D416BA6F6AA
:1052D000AB59048C107737C0B07A9881E7B7600873
:1052E0000477037FAF419BA2CB03BD9988625F38EF
:1052F000ED804010FF3434B280DB4E78F843F48CFC
:10530000EAADEC1E030167DBE8200855C2309BF4D0
:1053100056B3F00C800121AE063F2B6096DC200DC9
:1053200062D98831D305BB201C0465B30695FD0FF7
:10533000E8F9A1F37E7320D1B8847BE6230208D874
:10534000EF288AB3B4B6E72995661BB329F1FAFCB6
:1053500010F02001885805491381893AB4024406A7
:1053600019B93849622FB330011641DB2014F29687
:1053700026F5A860A7E9EB50193827199D1EC8012A
:1053800035BDE041A5DCFEF6C00378C55E193C885A
:1053900005B00512B30C900769C6909F1ADE70FA2B
:1053A0005396C1F09FEF4D1706C0CBA96015F2FAD6
:1053B00040D3416E666C1968D3BC28B366BE48B34F
:1053C00021724E4C88500F26C4845A169462F20FF4
:1053D0007FF608302BBEFFB915B309EC46C0488FE5
:1053E0005943165BB2DB20F972CC4023F51724AF8A
:1053F0000A0F9840AF23DA0220BD8A462AFF31DF28
:105400001FF491951018DC687ADA680C7B329042B0
:10541000647B98C4FD66F6B310D3D69882473ECE1F
:105420004EEE2AFE0DE7F77715EE7A2A048DC2FFBD
:10543000AFC064FFFDC8FB6E067F909871114ED11E
:1054400084815BAA3ED01E66BBFF09F7B3DD2E0444
:10545000497305FC9B14F8507CB26939A828B9FB44
:105460000BA001BFB4983085E5E91A40128080BDD9
:10547000115412EE666FDEFFECC27635B572ED5751
:105480000A01C76FF685ED191BF8CBB32694458842
:10549000E6E79031B0FB028826AA6A846DCA211E15
:1054A000666778FF01E62F57BCF03E720166BCC804
:1054B000F2B3FD0524DE9869EB3A51FF7F07CB324A
:1054C00040D4FD9801DD3C88E38BFB186FEF989C7E
:1054D00007E81E7B7C847447ACAB1912C563FDEBF7
:1054E000C6F2FA1ED11890BDF9A0C2B580E987B600
:1054F0004793F98BDDF06BDA886939BB24B40590EA
:10550000666DE478C66E89BF79F7322637FB0904E9
:105510007B98B0105E98FB180490002223765032DE
:10552000A9F8390171B3A65AF9789F1BC0279BEDE2
:1055300018FDF95DD16FED9834017B981A49B28856
:105540003D68FEF7673244063DD52239EE041ED38E
:105550000DB68AED13D0BFCE7FE4E0FBC8F3D2DAFC
:1055600033302032D0F761BCEEEE3267517952B35E
:10557000B0E70901846A1964AED6282E19B56EF514
:10558000986075A43DF310040218BBDDBEEEDD3655
:10559000DDEF9842663DBBB401CC9214DA9060FD19
:1055A0007F95ECDFB8FB54D9DE1012547FA498909D
:1055B000B5F62E01210AEFB396FEA2DDBB11FD1553
:1055C0006E71BB1C336E26E366448DF8FEC5D10CAC
:1055D0001AA6FAFB1120EF3BF643FCE89130600776
:1055E000590423B7627D15B6FF167503CFCF562D2C
:1055F000EF1172C002BF32226BDE2446C182C8EEB8
:105600001768F8D7CDEF3D98E4EE013C90F198F3A0
:10561000B7787866860A1316AE74B307290ED3A638
:1056200088C712C01D79E326C6F06FCF300C20D892
:10563000FC960426ABA602F9301077AB9808EDC2B1
:10564000F4C05AC4A93529FC30D70806CACCF7FBE8
:105650000BFD8BC47ED196F334B9A1FCA1DD1024DF
:10566000A4FC3D5E982B19D39858A26265674B80C5
:10567000046F992B8426AF04EDA109601DED26C0AF
:1056800088E78FFB2AE0FF77B09844189B66C8A490
:10569000B823B8C22409B5C7CFC8AEBAC1DD3B2113
:1056A000D8F6637BEB0887C9C01040ED03480C16A1
:1056B00098D0FAFC32E6A066CD1DFF1E412099AEBF
:1056C00070BB41A3EFE1725466DEEE7E96C0DC470C
:1056D0002530C1FDBF77A410FBAD5A22F3C8209539
:1056E0001057A510EB980357D158BA53B9EBF841AE
:1056F000E57618FEFA2B6FE0D69803BC302F413DBB
:10570000BA7A20BB58282EBEE3FBD7E58032FA18C0
:1057100040608DA433C8BAEEBF4CAFD7BE0D76063D
:105720008CFE4D8800D07B980B2A2DFC360FDFB005
:10573000B1343452FDEEF90840C02898B85BE089D6
:1057400080820712429044F5E060DA8CE7C8B8FA2C
:10575000DC57ABF8F513461AEEFA4C0A4E3714F341
:105760004002D357AF01F843A126E6127FB0980359
:10577000F2AF1EF798E8011CBFA0983081787A0F2D
:10578000682798CD9A1A45EB0B4001BED807020F47
:105790000553D3CA8016F6C0033A209DB1A330FA50
:1057A0005CF7D82048FE652EF9C88E02D7C04104A8
:1057B00097F360F57AA72F38441733E19F73D364CA
:1057C00089416D9BC880233BC8E9FF956046E4583A
:1057D000CF7FB9982105A0F385046145B39BC80428
:1057E00096D750BD83EF280104EA6476D523208440
:1057F000A7B39AE66FC278FE9710E0FEB960FFF19A
:10580000645104C039180240BF331C2C9B057389B6
:105810006C26E950764BF844EB1A2823E799D4C25A
:10582000045E787E5DC8B5FAF7F69CB38864E5C877
:105830002FF082F54E201CFA6605EC3C1AA6C0B388
:105840004D4D49592871CADD3A712BB751DE11BA55
:1058500019E8EF3F986E0665A10880E47A98202940
:1058600091ED70000F79A4AEAFA753510166113AC4
:10587000DDBB08CB10E0BFD6502FC0212090EB6BD2
:10588000CD0320F8207F9236F4D382326C360102A9
:105890007063236A270DF63190A704B3A61A67A791
:1058A00041AB45110673668010BFD4E5C0EEE446F7
:1058B000376D9FC80AE2FC045E98F706C228587349
:1058C000308481C70520CE02484408937D1A408465
:1058D0001131DF92FBAA96149705BFCC10D0DA7B6A
:1058E000BE53DF24961845B9C8FB46010418115E63
:1058F000F7B10AC8FF7B9807F00B1ED07E6DC84138
:10590000341257FB60B1605D3CDFAC8EDE1438B8FA
:1059100080190E4A078DD33810DF24C856B40CE125
:10592000031DDCA0FA1444F0C34489CBAF20B5D8E2
:10593000EA673DC9DB146BCB288A27F65461DE98F1
:105940002D6B7A0A72D309F9361401DFED28EF982E
:105950008A9089880324801F9810A1217537DC3133
:1059600040BBDA0154AFBF2A2E73013005ED092088
:10597000810BB3ED4BB3C821D2E8FAD29188B79E20
:105980008BF1DF98A14401021AE84012485CD3BFB2
:10599000B1A8EFD4FE41B801B43AFC7F24D7D412A9
:1059A000EF8BA0F298DAA8F2B5DD0342ED4658FF7E
:1059B000B65BC8F9987E6E18471EB6107B2FA26E94
:1059C00054EF9EF850572ADF036CB719E330F649BD
:1059D0008F893B17FCCC900131B7FBF598061DE58C
:1059E000E74693D02D7AE64AB30277C1042A992E6E
:1059F000D90701235101A9BF79E77D32BE4A7B0B4C
:105A000022EFB640F682819026333918F121BC028C
:105A100090BF773EEEEFE1EEFF320B1036A4D9EEE9
:105A2000921B019BD028224F690504287B6069DB0B
:105A30006432951941C7CEFB1284805D1AC71608DF
:105A4000AF98CEE814A51102FDE3E3EEF439F85364
:105A5000EE213ABD75B916C824D633BE98F9240490
:105A6000441803B3BD20B3E86B9BC8205CF5C84164
:105A70000C88EFC51EC0017A5B61699EA5AA0EE085
:105A8000300E73E30AB00BFA1C59D576A51F3AF510
:105A9000B75B77FB9828FA7FD11FC9A9E37A99C130
:105AA000B97D035FF94524A71CF9B9A6E8A8B0FCA5
:105AB000F2C3E9FEE06CCD2DDF4066D7C9F8CCA07B
:105AC0001020CBF55C23BC0B8829FEF422C08498FF
:105AD00080515CBFB30E098B96CE861BABB0129F74
:105AE000B3A00602289836F5208080569DD3F7642F
:105AF00035E62110EF4B340420C09A028392D1CCBA
:105B00009E38E910D01D4250207EACA0D35EFCCE62
:105B1000FFA7FAE7C643AC13D622A0D7E1E1B01A3B
:105B2000D10B9A2971A17A42B504CFC822E8FC7F33
:105B3000B7C6C280FD47FD677F8AC53934EA7983DD
:105B400088BE25FEF64FE03712BB8068ED6F94F8F3
:105B5000D346C1FEE5A3F960F402DCE0B85095DF5E
:105B600070FB7F81F930C6EEBAB6EE7AA823331BFC
:105B70007B56E208BBBC1880036E5E4AC0D378B582
:105B8000E023FB0C68B088F08ED3758A4830C2944D
:105B9000E84076AD65113532ABDC2CEEC4FF4B66C8
:105BA00036E6820930815E98FA18400360824E180A
:105BB00004C0C488886AD39A190A80E7303042400A
:105BC0002BE129E819081E30E4BE5847FB9809026A
:105BD0007EFD73AA17FE09DFCCFF870B2E840530EC
:105BE00040265ADA69BFEC90300124D7C404DF6341
:105BF000BA432018B3FA3C7A01342E504A7D0F0381
:105C0000FCC9325C0EC83B1A7F7B98AE3A143EFD4D
:105C1000982ACC0A02ED3DACE0D79BC893A5E03CA6
:105C20009017F040B506CCC81CA717B3300806B9CA
:105C300002D3016997D591E3EFFEE57AF096F1F88A
:105C4000ED9A0BED81F398FD21607F9A4E7D45AE74
:105C50008EFEFEFF10BD74465D64D68023817F9A60
:105C6000400526E0B4700852D329D5BB1768D2DDB1
:105C7000440BFEB9A026C2B51F0BD26281E0307082
:105C8000F6C0026D205DB221F8FEDCE69E26AE1A5B
:105C9000400A9EC1A2110522EE435D42F048140164
:105CA00020C07F37933B94FB9805D1BB0A3C4E093B
:105CB00010D22A42CAA82C929A8EDC08F0988D370E
:105CC00076D0BDFE36025FACB88126F3EAF669F302
:105CD000F39F1156AA97EE044FB285DD0BFFBF026A
:105CE00028C8DDDF9228415ADF7B35C8FDB910078F
:105CF00077DDD9E1482F01DF060410835F255F4F70
:105D000073B078BBD7B5EE1342B35AFFAD086DB789
:105D100007E0F6F049C69ADB0DB657C8D27F7D067C
:105D2000EDAFA3AFCC6EF282A0C8C19022B61180B5
:105D3000835D2F9BEFDBDE1053B347B33480DE105F
:105D4000D166BF11B306421D406C67EF0A68F92E99
:105D50009F0B3D1376E98C91F3C8CF2880A662444F
:105D60002CDE0408199DEE66EF10CC19CD1A04EE56
:105D700016466B4890573511BDC046C10880766401
:105D800002D3748CFC30AEA057301E969869C801BF
:105D9000F3F03DEED00338DE8B787D1E1B860CEFD2
:105DA000F9750508030FB3699DA8C803FC3DAE3C17
:105DB0005D2320C230469DB920A8FEDD9D79627921
:105DC000980AD6F3F2B8FEF56020EF3F8B8E85D0AF
:105DD000886E06A85FDFF652FAAF4BA9C16F20E7C5
:105DE000B9F7F8F20C40BA96EF67988821E426C418
:105DF00000135C22C6028CBC48662D802FD802148A
:105E00000EF4F2B9069C08DC4241B38E1257869A12
:105E100098FF2570FC2CF868FF9FB384DF83DC01BA
:105E20004FB622AA41772BFA8C0E61D3F847E2F9DC
:105E3000AFD919BD01F310641FF3CE30DF81DCEF61
:105E4000E192C2AAEFFF28FBEF166DD340F9363777
:105E5000C65F6388DDD7FC0173B36B29825FC6DD43
:105E6000FFA0FE2CE6A03466EEDDB1DF7DB346C7B1
:105E70001475208DABD31B803031C79098DFF7BDF0
:105E8000DD668FD9B977ABE520312CC1A3FFEFC810
:105E9000B2A0DFAE6737907BF39C7FB01D9EF822E7
:105EA0000A5807F3736DB521167B66CBF390BAB130
:105EB000F3514D962C7D5144AFED2FB279751946B3
:105EC000FA4124A9E3E6778D5999FD75FA920665A2
:105ED00018A88F98FAE7F7CCA8FF8B1AA43BF63DD9
:105EE000012DFB1C10554F08BA6510DB987118F88E
:105EF0000C3C59FF022DF4B8FDE6A1FDF9627E20AD
:105F00006CE2B2088CDE47BDC650FA02854678FFC7
:105F1000F1647D2CA99DF9EB6E19679892BF587BAF
:105F2000BB81E8FF6C9967118DB485AEFF1098FABC
:105F3000D841B49CF4B520464AA420CFF3E5D190D3
:105F400002D98AEE012DFEED1A48FC54B308A60DC5
:105F500028EC20F78FA94031016728B380DAB60218
:105F600083E523CCC1DC3BC359A2B3393419055AAC
:105F700041F302088A18E8481B64305AB334D60A41
:105F8000FEF6284004306BB3E028497534CA9758B0
:105F9000DDBD6B88A0A48222AB09CF03B3A1107032
:105FA000BFFEFFE18A69ED800CCF02101590220838
:105FB0000CC0E3504FA9C801216067FE332F9FBC7E
:105FC00014B9340442724121DC146EB50AD515F9B6
:105FD000E7018D22D502E0E758FF8BE0B730EF8F65
:105FE000F1D3608DB3BA49DF97D0080AAC82CB53A6
:105FF0003BE3CCB41B86F90181CBB3B6E3F5F98260
:106000009ACBB144E56301897B8A20F8629EAD5B3F
:106010002F4BFB0115DBC873E9311038B1FA16DBE1
:106020008040C44CEBE3C0B415CE5AE6FF75BABE4F
:10603000F6F70840FBE7679825F776B088FB6F6CAA
:106040006801552E10632613FAD2B3FF3E0BEFB151
:10605000C243AA0879FCC8B3FA795720373B08181D
:10606000F4F2BF08C45B8DC0FF12F56C069AC863DA
:1060700046F156EC96FF7FECF673EDD3FC1AFF3336
:106080004BCEE33364391C20622BBA08116C5F28B5
:10609000FAEDD8EA04EFCB99AF17DA64E3CAD6C9B0
:1060A00020C797F18B88F5149FB6054E4B319F465C
:1060B000ACE0FCC3DD6C15C0018F683D78FEA8C460
:1060C000B5D408618BA718FF61D26910CB2E89B3B4
:1060D00064BFB604629A28B00187BBF698FD1631FA
:1060E0008B8F589C80BAE3FDF38113F51D2085B991
:1060F0007C0390FD6EC363AB5D084F08CFCAF5DC2F
:10610000209801D860FFA28988C73E86C53D737874
:10611000D9FB08802298C79800FF3471D0FB3765FF
:10612000717FB96199B03E6C2022F598FE97BB67EC
:1061300008C5A9AC8F96685956FF59ED80A8FAD7C3
:106140000301FC928018C43F7C011DE55094B8D433
:10615000B1117F656760FED6A8E2079E319D78F297
:106160008F8C08623A7EB4101909FF02DC479981CE
:10617000CC69FEE6D8F80A88FA92F34F6E27189396
:106180001210020988F90965B6005ED04480F5DE78
:10619000F921BBB580019978C4FF400B0EA08E1485
:1061A00016820A0385EFAD269532FC0B1F0148804D
:1061B0000E05F3DA72306EE30C9040C250F0D3203B
:1061C00083617C059001C08AAF07D00A0243E1C316
:1061D000F8CF2022E3E8DA05A210D6F8809E302618
:1061E00082C117224062E16002094BA0F310EEB1B8
:1061F0000E109C2A2A40489FCAD21422445B0318DE
:1062000004E8211540570F5048FA647D6DA70C181B
:10621000EA2406BF752CFE77B24B08AE396EB74440
:10622000F598F8E90D41E879377E4F08FCDF0781E2
:10623000F2E446C40866ED225BD721F4CEB6EF6CDB
:1062400076A0FA5396A002EB7C012F764F0486E5E8
:10625000724C01D14BFA9702E7ED3497F44ECC6CB7
:10626000C379BAC6592BA6EBFDD14B0DFE3B765B2D
:106270001059931B40182041BE2EB8F904CE59D3B3
:1062800008DA7567F99498E2B74076CC51FC0A6257
:10629000DC40F2B03204406B330C2761FFFA635BE1
:1062A000EFA3024F75ED01B9E28B34ACB0FFE367A9
:1062B00018B8BFD8E2EB5E88FEAF02B04E456CFF67
:1062C000F8FDD09556085FEFDC06F1E18FB3033C93
:1062D000E1C5B462C5377B0167FDBC9C3FB1400D91
:1062E0006D42A8FCD60202BEE0B301F4CDDFEC7B28
:1062F000756750B1F89CB1E4FF33F25FDA38FD20E6
:1063000005265EAA6E239C8281D0083473486930CA
:10631000360670CEAEED6E4118805FCF2D9525F11B
:10632000B1D763818D26F528FF59EEED0320186D56
:106330009B8DFAE710BA3F5BE09103F3CDA670FAAC
:10634000729290DFF2D968DEFDD22CC4F403033CD4
:10635000B15AE5F1F80A62FB19E0F330F6A684B011
:10636000044293F3386605B7B05AD44C73D0224830
:10637000685F621E7E687E6BC99C22E070F364AB2E
:1063800078D3D695FDB6B32016CED48801B080D888
:10639000F358080BFA0C9B8489123BF39B81FC4653
:1063A00085C418F021236012BF8891302216C023C3
:1063B0005F79136021206CC13112FDFAE0413C800D
:1063C00007AFFC420FE0013DC0FAF0EE1EC0836C47
:1063D000F3813CE166E000BDD3E07871D322C6F1E1
:1063E0009CF3037AC9F3E4F3C726198008DBF44B66
:1063F0000CF37FF6510803A6F3726601BAEB8BE04B
:106400002F8F3846F321D36AF3F040FC8029806C4B
:10641000B3D14C82ED76AE190B29B3106BDDE49845
:1064200002B8B3C0EC61DA888021B358A3B3DFF3BC
:10643000A8FFB005046DB053103B789008C394F4E6
:10644000218D47EFF5B9EFAAC02382FEB518FE955E
:10645000430289EB9A82A0209F81B5FE676CF8DB2E
:10646000A8CCC6D7CF0237A32E9F4AA6815A72F96D
:1064700047D442778EDBF93CBA41CFD1C0A977AF80
:106480006FB1FAEBD4CF43F2984BC922F3CD24BDC0
:106490009888DC1101F785EF8ADBD0446A900239D5
:1064A000D6A644E006048DA49FD3F8FE0C88B0B7AE
:1064B00020F3989D2B12D0841A3B9C3019DE8867FC
:1064C000E3852933B60CF39897742828E01436DF57
:1064D000D89853FB8552C8B3581443A1E18041308A
:1064E000772402187E5204BF92B06819DCD10138BB
:1064F000FE3FB0E870800502D3D498A2D3AF844D9C
:106500009820D9187E322113BD9809AFFF3898CE54
:10651000BCD2BDA5E8E0013C882F19B88378B86DDE
:10652000ED980840FF30F6FE032807FE982DF87C12
:1065300098F4C679A1FAF319B5FBF1FF736DEBF28C
:10654000045F04B8D5E6142F7CF99F3EB7A8F1E5A7
:1065500024B50100E0E3C657D329FA10ED11310844
:10656000CBB3C69802C23320B3CB59FF2402B32861
:10657000D3D05816192FB308FD2089B404DCF310CA
:1065800037FAC5A1D3E21025D13011EF667DCACC10
:10659000EE5D44EDB3A2493930405EA0BF41A63262
:1065A0007782DBC5DFD979E59DB7AB7D6F999D1902
:1065B000882220FB8E63E411B6E330F256D3C5EC9B
:1065C000B5B72BB2B8AF6416438FFC30A3C4F32B1E
:1065D000C59864C0B43C9D13A6ECB56DF298524CBE
:1065E0000CE080FE363009D3FD1301B2667B98269D
:1065F000808248DFCFC5D0F0D7222076D971F64609
:1066000004DAF99837CD4821F5F493C930A86683A8
:106610003122B94665A34155E4859632E974F123E8
:1066200064C9B511E630148AEFF3AC0BA8A6B9849F
:106630005F7FEFC84898FBB3BF7FC6FFC020400410
:106640000B62820076F69C30FBBED219BF979892FF
:10665000B8F3785BC7F030D3860AFB5119ED6601B9
:10666000E27D98C87F2F104150D31ED3ADF2C1F602
:1066700010EDFD8480347BDFD498064D6DF61266F4
:10668000A5012673B78AE5B3EB135E5B300430D304
:10669000E8FCBB09B00865B32CCCE016C1066AB3B0
:1066A00040D5B115ED40019149B3D38C47E081F35A
:1066B0006AD35AAF85A024B602F6F74904B95D142F
:1066C000BB11D58909E2FA4B53F1874440D35423D7
:1066D000F84555EF959D0817A1DC73C22D30F4489D
:1066E000840840B9C16090FE12412048040938B2C4
:1066F0002ECACBC84F3CC5ECDF5E6444C05413EFD8
:106700000993D59740EDE86446FC1146F39CC81DFB
:106710003CF3F0F8808126A9E418ED5B3337BCA088
:106720007898B8CFDDFFF7D44452547F433C10E84B
:10673000DD3440E096CA189C654226FD8D8CB5FC80
:10674000E8AFFAB7CC5C688CA9F046188858116697
:106750001ECB64FB12444C540DBD9883EDD7032629
:106760001D44900288CE40292092FFF867524024B1
:10677000281F912012F1FEB780CE3160147CDA41DF
:106780003010C074BCB40B32939F660E30DD1080A5
:10679000EB053208EF8C614C80109F9216C0289850
:1067A00045A2B43E85D7F9FA9ADFFDCCB675F5B0AF
:1067B00020EDB81840FEB87B30401477F8BA490194
:1067C000C5D7E5E4D5CBE0D048F2A88BF3CB8B8ED0
:1067D00030F05E7F88FF8081306BD47D737FAFC5E2
:1067E000C1E3AAFC8B8F3CF5E5122065074B45728F
:1067F0006F12A576E01A3F5FD7D8801264F3686500
:10680000B311E0B9B3A3D31018F705037008AFF3C1
:10681000095EB3021802611D8AB66BD523E5220C0E
:10682000A79798F5EC018CD3B1EEFB1301046BDB59
:10683000CC01B2C8B930509342F4FE10F2012004EA
:1068400084F8F5B303CFFA92F7E1DD77BAC34012CB
:106850004219D3878DC880B4FE2E4E3D7BBB60BFEE
:10686000F9CCAAFE3F2CD08481DAA81901970799A8
:10687000A4E1B8442E5B1D649B80F78DDF76DC9825
:10688000E688FD6CA2BDE330BD070646BF4F6FB181
:10689000447C1B53ACF3C448B96F26047703102122
:1068A0005FB5C86C0FC9BB2D83FF807E8B2FC27E66
:1068B0005E304094F0410C0191D69326840A017316
:1068C000CB83BCEED55C227EA582480240130952E0
:1068D000DEC98A135CBFC838BBBAFA9B448045172F
:1068E00013C3277302F0208004184900BC2FF62F31
:1068F000333FB23E2E91E5D1E4BD850A487718B406
:1069000093E0CA9085E43F3CB717800339BBF84059
:106910000FBF963002BC5DEB72401E37A520798B0D
:106920007DA50BB3AC9E9103A5D11F8FE0E530C4CC
:1069300065A8A7846B3FF3D08378100F9EE8E60824
:10694000D0FADFD09803993E983A66400C5A40A09E
:10695000F52E093CE8646B97D5E5F5FDDE2DEBB42B
:1069600015E7F341FB1047261BCFF35D4660DC08BB
:1069700019D3AF2C6CB88208AE5E3025B3E716C0D1
:1069800002C088605E9832AA05B3C9F71E98FB2042
:1069900047A2E9EEF9C8DF8084A5CFEE8B428004E0
:1069A000D78430B3AF8FF1C366DDE5B62050BBD1DD
:1069B0009B82E981B32B260D1795EEF30D6C8AE8C7
:1069C000F9DF2E9BB242B820D8B39DF833A8A57D3D
:1069D0006EAFC4416BE7A5F912B670C838FBCBDFC8
:1069E0005CBF0BA8AEDC8BD3CFB822CCC374B3543E
:1069F0001081E4F227EAE522D6D728C816FF00A5C1
:106A000097C680F98B31F348FB037FAF9802E130E2
:106A1000DA2913F4585D476ACB44F266777CD26F6B
:106A20002EB5222B295CC5C80A7F9AA591845BCC20
:106A3000F331FE1951E19846E518B793E4C8D6A69C
:106A4000467F7B018360040C84EF1130821A9966C3
:106A50004177F835DAAF0C81D3C03918979864BC08
:106A6000845A31061F455C136122205CD0EB022959
:106A7000FCD5D2909BC81EF3C8E2AF01D7697496CB
:106A8000B85DC8E48BC47966CF49478DA50497E00B
:106A900010F030B6E0F2984AC6C8F3E230DFE9C839
:106AA000FF845E9877DB1FE5C836371804DF12B421
:106AB00004F0E5C5AE28F5E5F5D75A150160E07C90
:106AC0006D728ED8D3BF7F1184B0D9B34CFF8201D1
:106AD000384116C808596CE01505B3706454CDAF41
:106AE000205A9809B5B32161E478C0A514DF212E9E
:106AF000D3087BA6B0FC2005FACD8FFCFC2A04A2AB
:106B0000372B7BA74201A009BC98F383DD199B6456
:106B100099FDF2BDD0CF20EF40A005F0E703D70BE1
:106B20004C2BD6B4ADEDB3493C98FFB2E0B336067A
:106B30006BC84C2C1225EFB4C7B8FF77BE03011AFF
:106B4000B9FABF80D3C08B6138F919B390E67FDA08
:106B5000D6F3192240A306ABB6ACD3CEB827F4DEE9
:106B60006384ACBFA4C185F92004C003EC1517C130
:106B700050AEE037F030FBFBE8FF8804FCFFED3F50
:106B800041DD980146D01E0BF35DD97A662AF76481
:106B90002B9975971BC5EC98DC7150DC0DF91FEF34
:106BA0001A21A0E0309F0AE0F8804134E186E65CDB
:106BB0005D278CCB30068320181CC5DA6023F32CAC
:106BC000B4613F66BF5CC840E08511873016314232
:106BD000585726102C80301D267F7205804CD38498
:106BE00011D69C1857C81F3DC530E5C5E7E2F050E7
:106BF00006BC50B2087FCC5FDA0D417230F1EE4D29
:106C00003079E0E4C8C6F21B06C05F2D6B2F6232FC
:106C1000983CD25DFAA642BC506BA4FC346DC65DB4
:106C2000D9C859D56F94E80AB503F68BB8FDBBF8FF
:106C3000086CB3A62C191116D361E3F68C02299ABD
:106C4000AF6A669601D680B32D140193DE91B339F5
:106C5000E72261D377312388FA1EB545A0AA3149CE
:106C6000F65FA1248988D4423DFB843401A1B5FCA0
:106C70007DE0C03E503B53D926FC1AA551F70DAF1D
:106C8000A7C09AE16C01AF2D1B8B66FF3B2FCA5A40
:106C90007810A82008DDB5A610A783B24FE211D75F
:106CA00088029AAD69EEDE907F1EBFD35C7C5E8B5E
:106CB000DAF8FDF11D1250C460ED2F74BC00D98DBF
:106CC000E13B172402099FF8CC3B507D4877253DD6
:106CD00021FB75811FC1C758F94C13CEF390FE0AF2
:106CE00010D34FFCE53030DD76C5D1826AD87A5AB0
:106CF0000A0F4A1011767CD022A50228BFE097BC6B
:106D0000052D6522028B4C44F4143A02F48BF8EE04
:106D1000B3118172805804A3FBBB37B1D7401485EF
:106D200098C20B60EB0C84056FFC1466B319FF4727
:106D300052FC5088093012E740C102B390608014C1
:106D4000EE5DDD26F97F23B35E3E3B6C78FBF2C837
:106D5000DB9530E4C05D1D9BE8835F5AC5047DCCA4
:106D6000DB80FBC427A505E8F3C8209A1EBD781B6D
:106D7000D3F390F8235ED3C6EB0840FAEE125B66BD
:106D80001865C8FE9865707D672848027F405EB62A
:106D90008CF29817E04699F33C03CE50F8FA310292
:106DA000D8B3FE015DC8B6046DB3201279300878FF
:106DB00011B931C0A49CC0CA108BDAE048FA4B501C
:106DC00078D3400A08EBD86B20F9AC6CFF8BB3B7D3
:106DD000E9227F76C201D86299E3D370FD77DB297F
:106DE000E9279CF344DEB3D70222D63FFBF22311FE
:106DF000281B6CD398FA6C94F2B3F3EB9EF82485BD
:106E00002AB1C71DD630F92C8F8B661ADEB3E42B5E
:106E1000D71BC71839A2FB8C267B662C5026511D28
:106E2000FDCCFAE680BB077ED941E2B384FEF1DDFA
:106E3000CA05E598B1B9E0C636E8FABF4C785117F3
:106E4000F5BC924479B3BF28FF24E0C54F1776E61E
:106E500089FF3035F6F9717F8E7FCC88FF669ECE34
:106E6000F16AEC46DA69B3EBED41529A330333DA57
:106E70002080F8C345FF0288B6EC98FD77DBB8AEFA
:106E8000FF12325ED6E9403A9FDB98F8999CC64BD8
:106E9000EBF80473B11F37B3F3F4B2A2C3250F0AA2
:106EA000B9F668FCB384137202310861A7EEC968B1
:106EB000FD7F90A23610D55F827929E0F2D8A7969F
:106EC0006299B4ABEB08992758FD784BE4015FC297
:106ED000A2816BE4E0E51188FD9016E9EE0B40E33A
:106EE0001E57624180086A593A6FA0F946A890C1BE
:106EF0000618B9C07928066163F1A2265402200061
:106F0000CCF166D15A7627EBFB185ABB0928495FAA
:106F1000B4B5E6661A0804640994B305079459FAEF
:106F2000D642407A9421208C4CE3B0CF4096B2C830
:106F300023F76EE41BA2E235CB54CDA27A459DD255
:106F400090FF12E28146D9FB9067F9E09FD6DF2DD2
:106F5000EBD5B14EAEFE519C84627DF1F98811E211
:106F6000FDF2C4BC81CDED8D411BED3666E0FB37F3
:106F7000F6127F58659AA140DFC84BADC5D6C4084C
:106F8000340DB308DBA658F833849E434B1016E249
:106F9000043108733ADA0B30FB59EA08AA340123AA
:106FA000E5A70BDBFF90FA65A8101BBA977C180DBC
:106FB000FFEDBE28CB52EF456CF870FB5DD310633C
:106FC0005F78B602FD310892D8F1E0FD8002D99BCE
:106FD000942C0A53C0A5B13C8A10C9FE9030FDC262
:106FE000EFB1E77F1D4BB2ECF88FF9B5851F74F652
:106FF000D8F902803FB6BA79AA8AEFB9A8FF67FD2F
:10700000988FE51DB7EC0681E6D6D0FBC4784DC25B
:1070100013B23056034F6EB990FCE3AF3BA1BEB143
:107020009DB1549FE57C60FFEB988E611EACA9403A
:107030004BCB2D6C96C296DBB9303E58C851FDFC47
:1070400010F8C6FB12F9A78FE6C8FE030E96FF8064
:107050005FAC7BB034EBFECC54F6F688FFDFF72252
:1070600004FE5340F20A31F3F36CD4D308B6DA0CC1
:1070700004B6F3C0FA1D9B19FF2D18014D7A70FE5E
:107080008AF5CEDA3D6536D1208039DB970296AE9F
:10709000FD429D40CAEA89CB1BC512AA850D59A0A5
:1070A000F8FFBE64ED94EABC803CADB2CBF5840839
:1070B000AFD1A387E4D3EFA3053677F360FDC079A2
:1070C000D893B04CE0245A2198524BB28377D59391
:1070D000FB23C392FDC98F303FAE48B4F4ED04AB3F
:1070E000C4CFACD94ED61D11D2699427DB68F905FF
:1070F0008D7939BA301265CB48DAB10BE6EB80AB4B
:1071000050EB44AE42E9B33E01101B7E8F77A8E9F5
:10711000FB4083F2124AF450F822CD130032C10B27
:107120000703286BBDC91640A1ACA3B3A0034963F4
:107130004CD93EB8A0A80DA5BFB050CCC00AEE2ACD
:10714000FCFDAC20B8FD80487006CA1838789390D2
:10715000188421F870086419DC86864281605A65BB
:1071600072BB01D12A1139FDC4041A2F5E7CE6CB13
:10717000281A1260E79229A8E20CE8D2F94074803C
:10718000E50B81118EC52DDE807FD12044E555674A
:1071900069E1949F25CA86BF735AE8FDF908708B90
:1071A00037B5C182409181DC7A7FD8D4C70BC73014
:1071B0007DC89308D864E443D110D128FA688DEED5
:1071C0000011F2BC338DFE2DCFF6D77CFCC63416F1
:1071D000BC61CED9E9ED493E30B579F4ABE0084069
:1071E000720A28040C1D70F8185DA6DE67752DC69E
:1071F000BA36C21EEFB108F8F35E3BB61808EB31A1
:10720000207EB0AD8734A9FC4D6201165EE45DA717
:107210006534050280ED5F15BF90ED0AFDD4045C76
:107220003568F3058F6D969FF698FDEB11C0B01A87
:10723000AF2B06FDF5FC96D1B5883025D1FF089619
:10724000FF9E5798E663AB58207FE51458FC168FD5
:1072500011D2548BF087B2BA551920A5FCF6AC6751
:10726000ADB122C8BECEFE3FD29BDA01106D2FBC5D
:10727000329E74AF6DF2847575F9B1421D5E87025E
:107280006201BFC0B3625F75B3103AECF3193BCD36
:1072900004F6C98C1073EC22FD6DE050FBC29AD04D
:1072A00062C2DF4E20AFB21308104D08B3A7F4CD71
:1072B0008BEE8FD975940CA049DD1E9008E4F30F76
:1072C000F6042278FF439C602064368203013FFD70
:1072D000340C84942FAD086DC7C8FF90E4C02570AE
:1072E000E0BFA49003DBB19523B37F6659200EFC69
:1072F0000D8DF13AD3BF8130ED1048FB49759E6882
:107300004788EDB724DE03F5A3A6E039B5286CF76E
:10731000FB60010D80106167F35F1F3BFEE8FE74A8
:10732000DB938E67FF3FE8D8D401446EEB7E39696A
:107330009136FC46FDAEE5903006B3A738B12C90EF
:10734000851B0620C5B37D3419031867781693E9A9
:107350000CF30F36F83C7267E097B007FA7F787449
:1073600043E401E0BD70F320DC0FE0F3B7FFF980E8
:10737000267A0208C9F5BD30897ECF06D019ED38CE
:107380003A7CF6F3200C9DE60810F9BF6F9F035B73
:1073900069807B8A22449B08B31139B3216EB35AAA
:1073A0008BD20930D814E5F3020EB3F3D8F8EC8988
:1073B00080125F431E62236FDF0842C65F23DF63D4
:1073C00021898480E9C29002E060160D5EB33BA380
:1073D0009B7BB61D3E12A88D19FE5FDF659BE69B69
:1073E000DBC40C23AB3072FC80DB85D37365E3F91F
:1073F000DA47F3FB9830F847D6FDF6FE98B4024D15
:10740000C916FD19C6DB7E79D8048110D6B9B2F64B
:107410001A37FDC22644C0E4C4FF2798FBD8FD0CF0
:1074200068CB7F9B9877FD9A04AF0BB1124E0D8805
:1074300016CEC02809130877D3A001F8BA2B41B89B
:10744000AEED67B5CBFAE1B0409E16FB18208BFF7E
:107450001498F3DE819888EC6081404F933AB266CD
:1074600081AF281C9B264C08269C63308660F92C33
:107470009081C6D749F9B8B2800730B71EF998AFE6
:10748000BCA51EC403780B0F114FB5E0E08807F0D0
:107490005FEC31E0205FFD9CF04021C61AAF7A9886
:1074A0001C0028FAF2B22FE31637B5FEA535F38398
:1074B000F69F25D567D29ED3EF2F6B35A57746185B
:1074C00010037D723B1749FC10C9B3C0085F756C8F
:1074D000B3CE0423E02C02C444B3330F16C110080A
:1074E000ED05136279D1C0D22250A61491B310EBEE
:1074F00070F23234CA03BF4E6A647030D1E00AA61B
:1075000088F3300884F4C014100299876801BBA086
:10751000DA2DD0886EF34801E530091719DA2CF519
:10752000EB92CA80035839970A7DCB069DF3F6B8D3
:1075300082DBC834B45FFBD264608FE55BB00C7251
:10754000D784B9300E627C339721B4E9E3173F1139
:10755000A5C7C27616EE033038D1FE082AAA8C10D1
:10756000223CD1F4EE58300D8F3930800530E4DC08
:1075700001026DDF142CC330C3189B090C12B83004
:107580004BE619C9B32D1364FE3F01B830E5EC0A90
:107590009CB3CA4130C5D87D6B7DBB200290C9ED3C
:1075A00044F3E6A34004A681BF39FB5EA55CE19CE1
:1075B00080538318A28C161A91E9C8FD220393CB3D
:1075C000302257F8F2013CFA8003702006E03DAB10
:1075D000CEA5F098151EED8B100F7023AE5FDAFE6E
:1075E00030F6BA61F24914F3B616B1103E123066A5
:1075F0006F27401810771F3DF77279ABA79798EF68
:107600002BFF2CC1B56CF398C5AF3CE504D6A46F35
:10761000177D3A4A0246C0CA5C6FB74C82E964A63D
:10762000DF1103B8E3B07B50F84D79B00440480354
:10763000B28A2C5FE3C93044A5D9412D276E9E4400
:1076400055E6020420751AB9EA14BD01EBD0C02832
:10765000927178DE51DB28F9E6C803CCE392CC7155
:10766000EFDACC12F5BEE6A15E6B05049B1BF8FDBC
:1076700055B306AE6DF50CBE30B4F8C492FF0CE6FF
:10768000D8968EC0F69814C8FE3B30D684FA80CCCB
:107690009FAD028102ABA5200B35D22CE6E57A5BCB
:1076A000489A3CC042F4B8207E2C8005FE5A1E9AAF
:1076B000E7C88008B59269194298B0146DC0306669
:1076C00005F344589287CFCC51B020268502800321
:1076D0008800AF243F0ABCD3100983AF509D7FB30D
:1076E00048F8AFFDA71E508078BFABA506CB8B8CAA
:1076F0003043FACC7280E303F830CCF198F3CEE259
:1077000041C6F8FFD033FF5BD210707D9644A928A4
:10771000FFBF0184505E9DE0D38241DE987F2F3011
:1077200040D615E1FFD7EEDB16B3A8AFB30801933F
:107730002059C86203B4063149B34820E80B6204FB
:10774000C0E2C6FADF3BC661E3EFC0FDF35AF9C8F9
:10775000602DBCB93D209A43B60C59B312BFCCA7DB
:1077600024B51690029F5291610C8D82A401D0D055
:107770005C42049FF2C62444B410D9C0FED9C8B7F5
:1077800010E3302B4C6BA6F84280EE92B1F473F309
:1077900098C577872FF3B82219F15BC070B67B06C6
:1077A000809C306EB06E0E3CCC0802B1C08F804D14
:1077B000D3C801E7C790A619C7F9F86ECFD990686A
:1077C0001FE55C300171309FE7987491E3324458B3
:1077D0002CED9B84A04066AE7000880485BB1182AE
:1077E000F9453E280966A1995E857E40C8479764A1
:1077F000AE16A697FC183FCDC080209808810B4498
:107800000604FC84C8EE57A04157B36DF0FB3C98CA
:10781000F150B0B40259261EDC306FFDA9401CDEC9
:1078200098AC0E87D50F6D97C8F323E881F63C100E
:1078300048FA9A4F5FD67E9BFCF13011A39C7D9C49
:10784000A1E0BF392F100806650DC696EAE6042FA1
:10785000D3F8E63010D1FEADBEEB94E04C2F6DCBEB
:10786000EA0113DEE310306620C28B05E1D3CC7F42
:10787000A998184F02812C099720ADB7661012FC09
:10788000218ABE9799167FAA0B021E8CE0B18D4DFE
:10789000BBB2C84CE0FD140F5A102062EE020C2857
:1078A0006E401404E5300CDC30EC40B4F9B3D2FA8D
:1078B00067E38EBAD10B12D314C52A73FB4979EF53
:1078C000FF4E69CD70B0FFFB736BE1585CF3BF07EF
:1078D000C598D0D9C8677CCCA5F0E304DE98150222
:1078E000E04946C06469E5B39C8130FFBCA7178BB3
:1078F000D78F6A3666F39812406751F82204C04267
:1079000098C426AEE00A3094FE9A36AE2244303057
:10791000DE59FAC0D0400866D7558CDD8CC9EB988B
:10792000A4D16181309FF0CC39491002C921B369DB
:107930000B60EC4833EF46AA9829C4C68084113006
:10794000B7FCA22632AFAD7F1A029B3C2E362F5DCC
:1079500031C52E7E7AE2013C9007F2EE623D7A203C
:10796000E9E401C6F277A19818BF95305094C86633
:107970007F97AA5E9E0F69F69F8676BD6BB544EF32
:107980001682013039E0C480E05A2269F2BFFAFF62
:107990002E6B9D64C621FFA019A6D3E0120CF32F15
:1079A00073B33819FC807BB3C85C5BF071F3DB6C9C
:1079B000C604585E6B45B3EB12FDBC763E1284EEF6
:1079C000533004C584087FE1640B6E122CD9510832
:1079D00065B8AB20893415269AC850F7580C813108
:1079E000E7B0A0065793201308210BA009C0340468
:1079F000B2FD7A87C9E43D8105B6E3E46E966EACCC
:107A0000962073BE98BB806B3CAD1E350840452F59
:107A1000F47FEA7F283072EDDF77AB19799875EF44
:107A2000AE5A838F5E441088072BD3953D79DD12C3
:107A3000013CDFCC8C14909302452360BFCD981697
:107A4000BA68E07F69107D0D46EA76D696C7602158
:107A5000C04558CF1368E0A001344AB302210C9B03
:107A6000CD3B4998FBB3D506DA8244F130BFF7909D
:107A70006081F1309DBA9608188B19591590C33062
:107A8000DF02E70A40C0BA092335EB2CF2FDD1BA78
:107A900064B2F5C9E53010DF22ECD0037A4F9030A4
:107AA000E0343D9070941EE0D3BB64FFDF72401E53
:107AB000C083EB38100FD77E2065C87DB9B1D3B72E
:107AC00038300880602C4F867DED20B803B2D5DCBD
:107AD000EEE17CEC7FF472C8F8CD5E98A38819FFC4
:107AE0004BA069FB4A0BD6B3347BB309225D0AC8AD
:107AF0000208E08DBE183F180203AE607D7C912025
:107B000010C8FEAF9325B768125C300289EEEF17FC
:107B10004103D04496226AB320698882750230F707
:107B20000A7D2C88053472C204BD9868D7014DEED9
:107B30007B21F8CC0CCCA196B3DDB38116BB08FF3A
:107B40002A2DC6B870942631547F8898EBB380C133
:107B50005068B3BFF08530EE0BDDB3CFCBC923D86F
:107B600067AF1830F0602885BC989AF3C240F4984B
:107B700020D76042F7D250FCB4DCD02472ED224210
:107B8000018B6685263993EB9810675E1020125B97
:107B90005A776B8401C698C0166EB65AF2980D6873
:107BA00040B7E0D262526644C0B0BCC6FEC3BA2140
:107BB000960293D982DB18010025A5221941DC0326
:107BC0007FB39810011D09860B731B8205D4A8642E
:107BD000E6C878036E2F302C98AFE86D98100772C6
:107BE0007BD7D7F5682FE032F57810DE9859BBAE19
:107BF000407C2378200FE041ECD3F0FCBCA3C8A963
:107C0000CB2AC598F31666DE66FFDAD8029E66D3E5
:107C1000FD801808036010B7DD52C723F030DA701A
:107C2000FB2DB308B9303069EE98236008960C3408
:107C3000DFCAB5087FB38448B02012C404A558D366
:107C400001A3B3C2809C58A640014888BD30126889
:107C50007DCC8D2DFF04FAE5C217FFF8FB202BCF5A
:107C6000CE85D254F35834F359FFABB421191DD348
:107C70008888F88D0B95DE0ADDFFB8FD248D1993F9
:107C8000E6A236D3D9C9FAEBCF0408967B0224D3F7
:107C9000ECE9F820F528108C2C1B20FFD971102C52
:107CA0007BB8F9465944E6D151F3899117FFBFDB00
:107CB0005D8D17F6C87D32823FF7CC98FF9B9AE91D
:107CC000B56543AF2F8D8832807D97087EDEA89EF4
:107CD000B242BC89B8823B4F6C2BB0FD7FE59483E8
:107CE000847F6E4D71E8FEBAF101C936C13170135F
:107CF0001929A202667F59B8FB01866BFF80758542
:107D0000119087D848FE9F99E8DF82B301F63D566F
:107D1000E0DB9E9DF3EFE6104088FE612FDECFCAC8
:107D20007ECB50FC63A03DD4FA19E4DAA66FFB4C7D
:107D30002218E3D9DBBD1240F2A151ABC1B0D81279
:107D4000F276C690FA4126EAFC043FDC437A91DFE2
:107D50001887DCD564DC8420D65F5B779E9FF4783F
:107D600075E8FD60F9FAF59848CBBB0CB7B4264C22
:107D7000A05009CDD688DA059AB39F60ED801436FD
:107D8000C033CE0661012BDE40AE22294EC61B9BBE
:107D90000C08FFC43254E04A10827F524008800130
:107DA00090227B476910FB40A8081425104C6631CF
:107DB00089963C252289BD10E80882412495782DBA
:107DC000AB4F24BFAAD8A2FAA532A3BEE9C7791F38
:107DD000017AFA10383742AFD580CBA0D4CB30B37C
:107DE00044F4ED185820056A939EDE042080C47F79
:107DF000CC1014BCFCCEBA67CE59814C3E4B652CDE
:107E0000C440555E803100021AFAD521CEE671B821
:107E1000F8F3E615DD60408C6E3C80C45B7D50FB62
:107E2000087A31CF231169301C1BDB86C0FA143F5E
:107E300084CCC46C57FEBC8DF9DD7198B0FB8F8C7F
:107E40009C754A026897D928FB0B8B092C7CC7F5D7
:107E5000B201621EC7B0FDB476CF6CBA10028FD8E3
:107E600032FE56B8B120ADEC77083895B308E7403C
:107E7000F5188C18B2D7ACC1182FDB963FEEAFE4E3
:107E8000700875DE1E0428F88C6EF2E031DE256B7A
:107E90000898AE67FF7DC0FF63FF922C0BCF584858
:107EA00008BBD498FA6177D635D803A0E6F69B24B0
:107EB000FA02167A5D10E0536C4BC7469A90FF6148
:107EC00059689E14B2027E1BC341B3C565AE312210
:107ED000F394F7EDFD68E161979902FE70D8D8F848
:107EE00059E69DFC05625F22B0F8B819B630C63E6F
:107EF00061C73A64CFF440420B18186CD6E0FB4BD4
:107F0000B68C2036A6A3407C24715E54E7BF406D3A
:107F100049CDE6F44658FDCEAD0E0417FB1091C1D5
:107F2000A6E6058DFBA8FD8EF52D8F8D07A904A96A
:107F30009A6962944F67720A88C5D41308E07094F6
:107F40003653CBB8F964258220A3A88C121B39D0F4
:107F5000628B5F104FF1FF0A2004D3DB02107358CD
:107F600012207BECD8FF4BC71046091140F3D4CE4A
:107F70004D58AE08901ACBD8843DD817084809450B
:107F800010592624BEEA3733C4FF40BB2069FCF8F1
:107F9000DA403B045FD3A0908103086DFB7BA052C5
:107FA00051539703E50680CF5014CB2A07EC030109
:107FB000A01B30209F36BE53610222766F7BFA727F
:107FC0000BAA4841D806092048CF43C9AE2CCF019F
:107FD000908888082072A50C8DDA58522080C2E063
:107FE0000CE2793850064087F9A829070081FE5F26
:107FF000A44A144DE7B55A28FAB220BEE78D600DA9
:1080000019F2588D43C81FB2FF8443DCEC8CD68D27
:10801000F6441008FDE4B6A46BF63BE2BC66CEF66F
:108020003B4008BF7F8010D7A712D1AC93DFCCB8FC
:1080300048ACE5D6C879E5FF6FB108AE22D8FCFBA5
:108040008B1ECF6324B0FF62BE58B18075CC04B1E3
:10805000249FED5F58FF986D6ED8B008C73A7072D4
:10806000FB3C1905CF583D0AF6D94BFDA4DAC8FEF2
:10807000185850FFA384D12F4FABF415086901E9BC
:1080800062B9C8631A4DB1449FEDFE78F93CF8F52A
:108090001901759393E6E839C7B8ACE0049E25450D
:1080A000CAFD187B4DFB94103FE838ECCAE5CAFACC
:1080B000A1A59AD9B780331596E6C025EBD54855CA
:1080C000A7F89C4263FEE8B1827DEC7B44FC63EC44
:1080D000037F37BE041B72A000205930A6B33FEACD
:1080E0000080FB5337EBB0A968B10338F5C0FFA09F
:1080F00057061EB972AE02456080AD44572F6036F8
:108100006149282BFB75104FDAB121FCB2A3CA38A4
:10811000FD88E8A0FE7B0DDAD580013CE3D551FB5C
:10812000F39FE2E1EDF5F918BF1A89FEED40F4FD89
:1081300098D31941F22240798D2BD30C883436EE36
:108140000FB880629FC6BC30B38B288D3D7562200E
:10815000DD0260DA17FED93CAAB4D0F6F88C848828
:10816000861E66EE23DE2443B167ADB750FE60562F
:108170007BDB387851B97F5C90E3F980302352C4BF
:1081800066EEF4E032062439AD01011B84EC0930BF
:10819000024BD25CC0B5FD8631F2B82FD374EB0C24
:1081A00088059D9FFE601C9001F273EA38209E0FA7
:1081B000F33C800374DB1EC43CF60FE0413C77EED9
:1081C000CC60778BF0201A21F40794D35E34D3046B
:1081D00009EF0FC041E2CADE7B06C2FF9A8093021C
:1081E000FDEF06CAE383768680813027DA64C03FDC
:1081F000E04597D3E96604EA9410D360FA88F94021
:108200001130F5DE24CD89118CC4E06BE9580423CC
:10821000D3882FE6F8E056059DC9D19815FBBF5EBF
:10822000AE8628A4D3EFBD27B348FBFC2008048802
:10823000FF6E0BD10A12E97A9810FF2FE35F988145
:10824000AC5BDC471DFC31CFEF7715FEB869ABBCEA
:108250000A95AC099BE8418DB73F91895FBD8CFFC2
:10826000505CBD911D6E1AAF3904FBD67D7550DE92
:108270002085E4CFCBF677D5EE864F586987F01589
:10828000F8FA27416401C24C43034072FBB217BEA7
:10829000FDFF88051D81EFDD5A8994A0A709F8C765
:1082A000775DDAFE447EA418F3012BB03D030AC6C5
:1082B000F5E5042368164D48BE03CAD82877B502F1
:1082C0000880E8462811370502B3DC6619F0F6C3CA
:1082D00076B57EBDB17E68A484FBC92757C609FA6E
:1082E00084D60810681444B73AEEB1893005461CAC
:1082F000A1760781207BAB1A60DCD1E0F8F5EE7740
:108300007C76B44A3CBF02B0808849D13C4B7508AA
:10831000FF7204FF310161F960000D80D007F0DDCC
:1083200024435E98FAA0013040062FE16E98011CAC
:108330007BCABC07D00F90F0EA23F417E0FA98123A
:10834000D7D7980C1AF88ED3C610688819F0DBAB13
:108350002EC5A5F3AF5737DE127E871C5178E4DBBC
:1083600003346E9308F3F05EEDE1181007D3C6787E
:10837000FF030522EF2006C1CD044275173BB382EF
:1083800008819FF14C8451300968B96A95AE39B7BC
:108390006439B38010A522F898A38649303FBFFE08
:1083A000200884889B06A31ABE03FF4E9804DD02B2
:1083B0004003F9300473CAFAA90AAAE7414E2039EA
:1083C000DDEE22E386D38A6BC0306DA0BB0881FD51
:1083D0002248A41098FF75B1E626F929B702FD5D81
:1083E00041EF191A2188AB73655E66ECB9FF11ADD8
:1083F000B62A38199622D97E5493F8C064063746B7
:108400001EAFB0E0F398C7D6CF8881BD20B322DC81
:108410000CFBA0E5DD66BD86AF9C98B3B5033CAC14
:10842000D07E6D41201060F8E2C751B318E5FED24E
:108430005B965B508213B930057FBDDDB225ACAFD2
:10844000FC40E56EF1FF9FE43F4E7F1E30B8BB5A03
:108450007FE38002053001CF18FAEE100240D3C24C
:1084600044E7600148A030191682A62BEED16B10AC
:10847000EE11796E36710DABFA4FA07EADFF01BFE4
:1084800089EF7F3BB386EA7901FFF83244208251BD
:10849000A7F5F9E0E0800C90DDF0FDC97840DE98AA
:1084A0005F2F171EC0BF03DB980C109C66328D0A2D
:1084B000777F139729DF0F65EB98404F5798088314
:1084C0006B01FF8F270CD33C08D740F8A83A2093C4
:1084D000BEF9BC6E88B60ABA6496B30CBD36961661
:1084E000F6BFBABB29AF03F3E52F8530F229BE8270
:1084F000C670EBFF80097953C048A368B3A4317DEF
:108500000210E88BD3770C2822B7B96A809CB1E6B9
:1085100064F94BFBB6D64008CE49C60288BD980424
:10852000D348FC9380209611E7DF64CE8042511837
:1085300051EF4698A8BB04DEB48AFAEA3AEFFEC4CB
:10854000547780FF100457976FB30AF7988005247B
:10855000AF90D7CC02E0920CE72009F98CF979BEF4
:108560001A58998419E86D9F042651EBD177F02AA7
:10857000D466F6EE04A7DB88E726EFEB67C82C6C21
:10858000B6E386F7EDA2F3ECF8304DF3161CA7978F
:1085900098937EEA6E74DCFB3C66F76D7698FEADD0
:1085A00094027D986059C85DEE5CF2A518EC412EEE
:1085B000ECFF7B6C241008018FDAE5301675A4FE01
:1085C00098470D3EC49653EF1211EF7B4B7686FE13
:1085D000284FAF753FCDC698E0128F5F3969214BA8
:1085E000D3FD80E620C2794033E211B029C108D71B
:1085F0008A08876EBD40320EEE70FB317EC31F7657
:108600001ADE8009954081C730FE32900D226A350E
:10861000889F19244C0240301799F9A6E01407B03E
:10862000846053359DE83C88722304DFC998F8863E
:10863000C612CA5A843EBB05820DE600EBCDC27954
:108640003064341E80E09B16B078F93008DC48F9BD
:10865000D81AC1FF86F3D3977DC07DEFF9C87FE1BB
:10866000970E5ECAF8B80646FE32FB7D98065FA4F8
:108670005E5E699D9BE1FE10E0C0A0A2536FDEE349
:1086800016C195F4A3CF3010112082BB02F0C4C2F2
:10869000E0143F6019698A01F044DE0809B3391219
:1086A00031228B7FA69882B3096BC6D0CB986035F8
:1086B000BD8F115FDBE18480209B7D505E39307778
:1086C0006EEEEEC3BACFE0C453A8A3BBF9FC98E1A9
:1086D000560FC505045F108C92F6F3110436E8FBC3
:1086E00088F6C2DFC8983DE37A27DE973EC9C38883
:1086F000E6475C5957B35B9692E10C11DF857CF33A
:108700007303E0FF720305FFAFCD75D2C001209661
:108710007CB9ECAE48A78CF7AEC9E782899FCF45FC
:1087200019BABB64287DB2D74BDCCF98EA4427FC4A
:10873000C64130081EFE46D92F191366C7B528C793
:108740009040A4186003FBCB24A00902BD972AEE39
:10875000F9ABE97BD0471186BB467A4490E262EEE2
:108760002D100A1D04AA0C20B73D829FFDF2301285
:1087700026015E725D51FF8C9009B00844C1222928
:10878000A8DF8442448E9EB3D8A3CE619FF8D71150
:108790009AFB908081BB2402BC1127BF8C21B58439
:1087A0007F192C02442012F8FA01723D05B2C8EE7E
:1087B00062300F60FA0C8003F0FD22837B98E48125
:1087C000E91C1004B3CADC233EABF64614CA1FBC36
:1087D0005A7FBC9803E2013DACF3BFF539C8C00134
:1087E000F8DF90FDEDD2C240C766E802DA97C2FB1F
:1087F0009888418A10FF4B982272D67F8AF9C86FF9
:108800009B9B045D13AFC6D320B4A12CB3B51D63ED
:10881000B3120A4DC09D02FC30EF1130014ABB4A31
:10882000B321F75CFD4EA2200422F7B340820189F8
:1088300038225F7247E48DD3E3FB7FC390465FDD50
:108840007FDA7F6B4C0812CE45A388492804023496
:108850008AF7C6ABCABBF330FFEA197CB7DAE0D0BF
:10886000F1307A4008DBC5D5DF7EEE90BECCF3F464
:108870002B8B30CDEF0FEAFC04720B4BF9DA50D79B
:108880007FAA9DB8D6D1F9C8B2103C8A4F19FCE82E
:10889000FA602DE6FC4CFE2230BEF50518D9C87BE7
:1088A0005446C0E9CB5081E475E84EAA9B94F33C52
:1088B000943603D6B89034F4A740731948AFFE1C21
:1088C0005A70D142A7F04A0C21284AE512FD88408F
:1088D000DD6C5B764FCE560DEB14A781CB5D3CB6BD
:1088E000BDF98BC2B422CA104066826C19CFA005B4
:1088F000B3A2FB80E591B040F4E38DAE829449F3DE
:10890000A29E104A600144068830EDF76A62A05FBB
:10891000007FEB577BBA4B824D837F328C33EBB0B9
:1089200049046DFC7F2130D6CAFEAB0F808F3DED30
:10893000B10FF9C88B220EFCC80378200FE4B9E60A
:10894000E990CB0ACAE69AB38FB0E21DF798F040DF
:108950000E7F17309D9D9AC81E1AA5C6C248D360C7
:10896000664EF3988B40D74E82E7C880101F036194
:1089700027931430807FEFEFCAD51C051777995BDA
:1089800059C828CA458D96790321B9F8B344BCC0AB
:108990000719EDAE8907300887980A5E8BDE8101E2
:1089A000B3EF0E404A77B303201381B3DBC81467DB
:1089B000C818056EB32BB5CFACC9C8F969C430C4AB
:1089C000EB34904042AF59121C30F78C77CB323BDE
:1089D000F863BF53F830E3E05F5E98347D5F2211A7
:1089E0007617B406E8F9FE374A17FF26F09D8E9FEA
:1089F000DF903048374BC0FFDC3713AFFBB41A347D
:108A0000E05ABA30A8C620E998AD30FA0FE385CF16
:108A1000C6E130FAEF22801E5A91483D89CE18DB1C
:108A20000DDE90EB69371B2D9BF25B57095C77C815
:108A30006AA75DC7D3F8FD338026DBD1827130276A
:108A4000B4D0E50523157330858073D35EB3AEEAE9
:108A5000A77E09F737FFD1069018AAB3418D66B5F6
:108A6000A120BF01DE47FC8081B018403F9ECA01B3
:108A70008C9045BB24C1E9284004C1440C57E67BD7
:108A80000A407C773D3F7FCF4BCEFE11EEC80218E7
:108A9000D6AE4C0868B321F8BC677A7F4C8021D3EE
:108AA000594F3798E0301E1C900320DB2BC88930CB
:108AB000E98EEE1A823A7EE1532F0B3D6040EF6D56
:108AC00098201E7D983C7F5F54EA5EE2F79888F814
:108AD0008477B698C120FC309420B6006BCB300868
:108AE000F830BEFCFFDBDC0BEAB408DB20C83F86B5
:108AF00030190C7D9B301068FEBE5E88B3F32118E0
:108B00000102E3190E13093936E6B09FA4B421E639
:108B1000BCC40A6BCE85B84508440FEABEEA64FBC4
:108B2000E24FAF1F439820D7B0FCE63B90FC02EF2A
:108B3000DD4114DE1302109427424813057998A3EF
:108B40007AB27DBFA27EDB80DD4BFFB8630BBE0A2D
:108B50008E472C9DAEC8B8645700FF812410C4FF17
:108B600069F69ABF1CF604403008862CBEBF9F05EC
:108B7000FCD6C42150A745F484DD0ABFFFE5577435
:108B8000BF9AF1AD19601AF3D0F900239730041F92
:108B9000C591C849919569E798BDA7F877A2BEDB52
:108BA000E2F78EDD5BFF97EF2D9D04CD9074AF7CD7
:108BB0009A412010F0A74653161408B803DA4AB5B4
:108BC00025D2B1CED10B04BD98051DEEB34448119A
:108BD000EFF32A86DD46B310BB022D0BB830FD82C1
:108BE0006B99A64401F73A6F4BFBD79C0640C2DD58
:108BF0002018BFA08C90513006260C88D6DF135762
:108C00007BDD52FFB5FCA4FAA3DC100119E1DBDF28
:108C100008A1C0E205CDB18C047998C75D7F328C84
:108C200002AD50DF9DFAE298AABCC55FB0EC980790
:108C300070390E117E6EC83CCFC8B04F48940B6F90
:108C4000B3C60D42BB683DC8722006B78D98F302CB
:108C5000E5C695C8EE8B10F980FF2298F050400CC5
:108C600059C5D6C037F303E5F5FC7DAD1252155852
:108C7000B3019AEB0C412EBA3546E3307EBF57DC88
:108C80005E1039FDA6FA26C010E0B366ED09577CE8
:108C9000B98B482021C2EF4C8809C99BFDBF44E233
:108CA0006FB82E90F0160DD308FE9845CDEBF55811
:108CB0008B1930C8317190FC58D9FF3DD79403C44B
:108CC000100032F6E2AB40FF38D3D7BCFBDF32E70F
:108CD00078F1759CF37F3966804422ED48B3EA7BD6
:108CE000EE281B60D3D0FA31E7FF980A55BB62BE6D
:108CF000FEE0EF28EEC6CBD736C8243C66F71857FF
:108D0000AC373DF8E4EE946E8E313913FC19FFD97F
:108D10004BDF2125F018DFA04CCFC9EACFB876662B
:108D2000ACD5209EE0A91022EC89F94D4F40775A2E
:108D3000F0BAF4942BC8DAF4FECC0FD8BCA581733A
:108D4000B40073D0BC8DD39BCAD8FC3C51EE35E83F
:108D50003DB186140248D57F58689E71B1A6D11ADC
:108D6000A4A9B1EDF399F89C0679D5B1F39C4E67AF
:108D700099D323B5D388BCFD0DCAD5100175C4E7BE
:108D8000C79882DAFF08CC2DDF9BE3A6041331D607
:108D900043EA7DB3464F7DE5A0FA11B34992BC6426
:108DA00091BB4389FC40262857D8D8F8A06D46E2ED
:108DB00087FDFD320D779D06647D0B98AAD818FDBE
:108DC000BFEEEF0A30C3ADFF5096F9876B338008D2
:108DD0006A2E635F86627FF7B4B8F54B11AA1F0154
:108DE000E3D9FA290B1351684009CB0B028195B7DF
:108DF000068D8BF45AC688FE3FE14E176BF80421AE
:108E0000F68080CA688231ED2169C99608CFDF23D8
:108E100059C528CF7CBEC0EE7D304504A0B426CF16
:108E2000E7C84003AC030C280226078002504B5EC3
:108E300068101415DEA09930E158F94438A844F3BD
:108E400051E6320A1BF50D0E91FC1F287004FF90AD
:108E500040A8082920450A90B19DA888DEED7E7CB7
:108E600001088134205ACE566A018F1DE01802078E
:108E70009120E060D0ED04843EBDB63D9C62A8FF29
:108E800082A3C57E6F3247D2260183C53D33084693
:108E9000717FCDABC6786E76058FE45FA040F4A7F6
:108EA000DC5A6B22196C0240DEB7B2F592047D5693
:108EB000AE47496A7E73BDF1FC657D168FF6728000
:108EC000CF37A527CD79B0F940DF0128E7D2916EE1
:108ED00025BADB02C6BC95C4FB5E78B3FDCD04C2E7
:108EE0009233C06F3DE5186BD6127FB7C6C0FC9AAF
:108EF000EFF9A498E26A4F614308CCF9651F68FB5B
:108F00008188FE4DC7FA68576119FFBD64B1FF1F24
:108F1000D8AD01EF5863B39798FC469D224DB082BF
:108F2000911A0865FFC330FDB302868BBC12DFECDB
:108F30005AA3CE7EB371CDB2FF7FFD6BA69E7EDAC3
:108F400066E98494087E981AB6D74AF6EBF0F97170
:108F500099E66327B61023DB58888DCAFFA148B372
:108F6000FC0C1B534CB17FEF7609B2F8B1FF3F0AFE
:108F700030C215B702A8D906E9578866608CFF3D54
:108F80003498FB109E2963EB1901156CDB98FE6089
:108F900096C2F16466671BEEFFF808017E98C55122
:108FA000D0583628FF171B81AC8F01FFD827D86611
:108FB000B3B10505EDA0CBA1F91158D42087581CF9
:108FC00045E6D277ACE520FFDB84C018E6424FEEE1
:108FD00090F94037C36CD50281EF331CFE7EF395C8
:108FE00030F3B475FCD987F9FEC46A797E6D9908AF
:108FF000CCAC22E72A48FD2064AF1C013C63A4C42A
:10900000BED18BA5CCD1FDB74A6FBE88FDE3A827A2
:10901000749E40DD68F5059E7D8E80D1A4226CE8AB
:1090200019199F0E36B8FA4263C7203CF482E8B2A1
:109030007A1AB61DC63AB6BFD9041C91BBD54BF6F9
:10904000763154FB0681106FF114163CD5DA1B35CE
:10905000FB12A6CF29E509970A24891092907ADE9F
:109060006E40218CFBEE0321FF836005E630011486
:10907000E918806E4E04ED200C36148263B50AFDAB
:10908000438980010895C69DFFFC14F0ED06186029
:10909000FF2C286C950030EE800440FD0C203F36FC
:1090A00028F880629008DC82400A0F1814B98021E9
:1090B0008419CCCA164CB1651F7C31600612803011
:1090C000859F201708011D22A8411C6406600388A3
:1090D0000532C770B371032001037FCBAF9B27F12B
:1090E0003D04D8B6CAEB8D3719FB6D21F3A8BDFC42
:1090F000E5017989AE6F2340162BDE29D91C08E0E3
:10910000472D6A92021BCBD8E9A5C7424AEF68DB1C
:10911000E31CEDD531AF6C370820E615D4FCCDF556
:109120006304B797E6D1720A03F06A237A8D060BBF
:109130003FCD4C0E38D656E8F95BF717678B7EE1CA
:109140002D5A20657902E6DD39BBD6FA14FB9C1C4A
:10915000CDC70898D56E26AEFFB332795560467EEE
:10916000503BB51231C87FB5A4ED9A38891966868F
:10917000167EECE44059D4A8B3F957DC047EEE0A1D
:109180008CFB436CA57DB168B1FF4F82F1C29D326B
:10919000A638ACFCB1C841355B672C6201F56C1098
:1091A00094CFBFC8EDCCBDE1028C80D4E5FEB3A066
:1091B0003F87047F910FFD8BFB42B0F879B4A7DBAA
:1091C00071ADD9440CAEFFB17B3F5A0160A6E708F0
:1091D00066FFCFFBCE75B9089AC763FA04EFC0FBF0
:1091E00002DDAD20A213087D342110440275F42C59
:1091F000E98047B74A04A03CD0E50920D312C790C4
:109200000297EE300CF321189166C1758481BDE49C
:10921000024A3AE401280447D01023B0A3F33DB436
:109220008023EDE004C117E107904CC60494C9C641
:109230000AF2F412019754FC17931112E311C3F3CD
:1092400071B0E6F318B6FF30F82AE76111AD9CE083
:109250009E18B314800272660A401F1E05A080F398
:109260005E50F30304900212033FBE1616C002586C
:10927000070BE001F32C8005B0F3406CF3A107F37A
:10928000B9FFE0FDA00C94813255FF06CA401930A9
:109290000365C03CF3993250FFF38019488369306D
:1092A0000DD9A641DFCCFF0C9001324006C804F373
:1092B00019200364F3A4B54153F313F31401E3003D
:1092C000F9FFB00811241FBECFEFD0E1DEBFCDBF44
:1092D00011E0A0E0B1E0EEE6F3EB00E00BBF02C06E
:1092E00007900D92A632B107D9F71AE0A6E2B1E0D5
:1092F00001C01D92AB3DB107E1F70E949D4E0C9459
:10930000B5590C9400001092620110926301109202
:1093100064011092650110926601E8E6F2E08FEFB9
:1093200001C0819392E0E337F907D9F7E4E7F2E06F
:1093300001C0119282E0EC39F807D9F7109273025C
:10934000089590919C02E8E6F1E0E90FF11D808319
:109350009F5F90939C02089520919C0230E02F5FC4
:109360003F4F4091610150E081E02417350709F03B
:1093700080E008951F93182F8F3799F08A3789F46A
:10938000662389F4ECE9F2E0129282E0E437F80710
:10939000D9F70E94AC498823B9F48AE70E94A14911
:1093A00013C0662389F0E12FF0E0EC58FD4F808177
:1093B0008823E1F0815080838823C1F40E94AC4966
:1093C0008823A1F4812F10C0E12FF0E0EC58FD4F6D
:1093D0008081982F9F5F9083882341F40E94AC493D
:1093E000882321F4812F80680E94A1491F9108954C
:1093F00081E020919C0290916101291380E0089501
:1094000090916101E8E6F1E0E90FF11D80819F5F35
:1094100090936101089580916101E8E6F1E0E80F21
:10942000F11D80810895882321F010929F0281E030
:1094300005C08FEF80939F0280919F0280939D02D1
:109440008FEF809367018091A50284608093A502CD
:1094500008950F931F93CF93DF93082F8091A50258
:10946000877F8093A502C02FD0E0CF77D070C13026
:10947000D10521F0C230D105C1F40BC081E46FEFFA
:1094800040E00E94784A182F07FF12C00E946E57D2
:109490000AC082E46FEF40E00E94784A182F07FF6D
:1094A00007C00E944655682F04C06FEF10E001C04E
:1094B0006FEF07FF05C080E440E00E94784A13C0C8
:1094C00080E440E00E94784A682FC130D10521F045
:1094D000C230D10541F404C0812F0E949C5703C0C3
:1094E000812F0E94D554DF91CF911F910F91089544
:1094F0000F931F93DF93CF9300D0CDB7DEB7C09803
:10950000C09A4A8369830E94C052182FC09869810B
:10951000862F0E94C052082FC09A4A81412319F019
:10952000812F0E94294A802F0F900F90CF91DF91B9
:109530001F910F9108958091A50282FF17C060913D
:10954000670182E24FE70E94784A60919F0280E2C1
:109550004FE70E94784A60919D0281E24FE70E94A6
:10956000784A8091A5028B7F8093A50208959091FF
:10957000A00291702091A00221FF02C038E001C03A
:1095800030E02091A60222FF02C022E001C020E0CC
:10959000682F647F692B632B622B80E54FE70E9465
:1095A000784A08959091A00298279093A002809104
:1095B000A50286FF02C084E001C080E00E94B74A95
:1095C0006091A0028EEF0E943E568DEE0E94F24FF7
:1095D0000895DF92EF92FF920F931F93182F062F9B
:1095E000F42E662319F4833809F41FE7812F602FC6
:1095F0000E942859D82EE92E0023A9F1113701F134
:109600001C3721F0113109F093C079C08091A60276
:1096100082FD06C0FF2021F48091A60284600AC06A
:109620008091A60282FF84C0FF2009F481C080914E
:10963000A6028B7F8093A60280E00E94B74A78C082
:10964000FF2009F075C08091730287FD71C0809181
:1096500073028370833009F06BC08091A50280682B
:109660008093A50271C01935B1F11A3578F4113122
:1096700009F445C0123120F4173009F059C049C02F
:109680001231E9F0143109F053C02FC01D3748F4EE
:109690001B3708F048C0173761F0193709F048C088
:1096A00042C01E3709F044C0FF2009F041C081E0EC
:1096B00003C0FF20E9F582E00E94D24A39C0FF20B2
:1096C00031F48091730284608093730231C0809181
:1096D00073028B7FF9CFFF2021F4809173028860A1
:1096E000F3CF80917302877FEFCFFF2021F4809129
:1096F00073028160E9CF809173028E7FE5CFFF20F6
:1097000021F4809173028260DFCF809173028D7F9C
:10971000DBCFFF2021F4809173028061D5CF80914F
:1097200073028F7ED1CFFF2019F4812F0E948B52BC
:109730008D2D8F3749F06F2D0E94BA498E2D8F37AE
:1097400019F06F2D0E94BA491F910F91FF90EF9071
:10975000DF9008950F931F93CF93DF93882369F5CC
:109760001092260188E2809328011092270110921E
:109770009E020E94834984E160E00E9428592FE7FD
:109780008F37920781F081E160E00E9428596FE7EE
:109790008F37960741F081E161E00E9428597FE709
:1097A0008F37970721F4809173028F7703C08091E0
:1097B0007302806880937302ADC08091A60282FD1F
:1097C00006C09E990EC08091A602846005C09E9B33
:1097D00008C08091A6028B7F8093A60280E00E9441
:1097E000B74A80912701882309F06FC0C09A10E022
:1097F000C0E8D0E008E04DC0E0916101F0E0E85938
:10980000FE4F40814A3759F40E94004A10922601C7
:1098100088E2809328010E94834911E03FC0809133
:109820009E02882369F08091280187FF09C047FFC5
:1098300007C08758823020F4842F8758823070F513
:10984000242F30E0C9018F77907027703070FE01AF
:1098500002C0F595E7952A95E2F79F0133E09695CA
:1098600087953A95E1F747FF06C0FC01EE59FE4F98
:109870008081822B06C0FC01EE59FE4F209580812D
:1098800082238083409328010E94004A00939E0215
:1098900011E00E94F849882309F4AECF809172024A
:1098A000882369F0E8E6F2E0958180818927182B0A
:1098B000919322E0ED36F207B9F71092720211236C
:1098C00049F186E08093270125C0815080932701CC
:1098D000882389F090E00197FC01E859FD4F6081F1
:1098E00060958E599E4FFC018081682B80E14FE787
:1098F0000E94784A0FC0C09A81E10E94C052C0986D
:10990000C09A282F30E02F7730702115310511F0E3
:109910000E94294ADF91CF911F910F9108951092D3
:10992000610110929C0280E00E94AA4B80E360E0FB
:1099300040E00E94784A08951F920F920FB60F924E
:1099400011248F939F9380912B018F5F80932B0124
:1099500087FF1BC010922B019091010180912A0179
:10996000890F80932A018F3F21F49F3F59F481E0B2
:1099700005C0882339F4913029F48FEF80930101D9
:1099800080932A0180912A0183BD8091B80A8C308E
:10999000D8F48091B80A8823B9F08091A50284FF99
:1099A0000AC08091B80A8B3031F48091C50A8431A5
:1099B00010F41C9A14988091C50A882329F080918C
:1099C000C50A81508093C50A80919E02882329F0A0
:1099D00080919E02815080939E028091C20A8C30B9
:1099E000D8F48091C20A8823B9F08091A50280FF43
:1099F0000AC08091C20A8B3031F48091BD0A843153
:109A000010F41D9A15988091BD0A882329F0809141
:109A1000BD0A81508093BD0A9F9B04C08091730250
:109A200084FF06C08091D90A9091DA0A019606C097
:109A30008091D90A9091DA0A969587959093DA0ADF
:109A40008093D90A80912901882389F499B3809160
:109A50000001892380936D029E6F9093000180E145
:109A600084BB8FEC85BB84E0809372022AC0813076
:109A700049F499B390936E0284BB8EED85BB10922E
:109A8000290121C0823041F499B390936F0284BBC5
:109A90008DED85BB81E015C0833049F489B3809397
:109AA000700284E084BB8BED85BB82E00AC0843009
:109AB00051F489B38093710288E084BB87ED85BB44
:109AC00083E0809329019F918F910F900FBE0F909B
:109AD0001F9018951F920F920FB60F9211248F931B
:109AE0009F938091A50284FF2BC08091B80A81507A
:109AF0008093B80A8091B80A8823F9F08091BA0A55
:109B00009091BB0A80FF02C0969A01C096988091FE
:109B1000BA0A9091BB0A969587959093BB0A809359
:109B2000BA0A8091B80A8B3011F48E9A2BC08091BA
:109B3000B80A813039F58E9825C01C98149A22C035
:109B40008091BA0A9091BB0A969587959093BB0A2B
:109B50008093BA0A869B09C08091BA0A9091BB0A89
:109B600090689093BB0A8093BA0A8091B80A81509A
:109B70008093B80A8091B80A813021F41C98149A15
:109B80001092B80A80E188BF84E18093C50A9F9152
:109B90008F910F900FBE0F901F9018951F920F92EC
:109BA0000FB60F9211248F939F938091A50280FF8F
:109BB0002BC08091C20A81508093C20A8091C20A50
:109BC0008823F9F08091C30A9091C40A80FF02C0F3
:109BD000979A01C097988091C30A9091C40A96956C
:109BE00087959093C40A8093C30A8091C20A8B30F0
:109BF00011F48F9A2BC08091C20A813039F58F9869
:109C000025C01D98159A22C08091C30A9091C40A5C
:109C1000969587959093C40A8093C30A879B09C041
:109C20008091C30A9091C40A90689093C40A80936B
:109C3000C30A8091C20A81508093C20A8091C20AED
:109C4000813021F41D98159A1092C20A80E288BFD3
:109C500084E18093BD0A9F918F910F900FBE0F906A
:109C60001F9018951F920F920FB60F9211248F9389
:109C70008091A50288608093A50280E488BF8F91BF
:109C80000F900FBE0F901F9018951F920F920FB656
:109C90000F920BB60F9211242F933F934F935F9324
:109CA0006F937F938F939F93AF93BF93EF93FF93A4
:109CB0000E94025780E888BFFF91EF91BF91AF915A
:109CC0009F918F917F916F915F914F913F912F91D4
:109CD0000F900BBE0F900FBE0F901F9018950F9313
:109CE0001F93CF93DF93EC0107EA12E0F801819113
:109CF0008F010E94C0522197C9F7DF91CF911F9128
:109D00000F910895F8948FEF80936500109264008E
:109D100098E09093610093EF93B912B882BB90E200
:109D200091BB9FED95BB14BA91EC98BB97E897BB9C
:109D30008BBB1ABA80E888B90895CF92DF92EF9270
:109D4000FF920F931F9333E7C32E00E41CE028EE2D
:109D5000D22E9AEAE92E80EFF82E0E94824E0E94BF
:109D600049540E944C580E94BB528091610081600E
:109D7000809361008FEF9FEAA1E081509040A04066
:109D8000E1F700C00000809161008E7F8093610048
:109D9000019BFECF8CE892E0A0E0BB278093A1025C
:109DA0009093A202A093A302B093A4020E948753AF
:109DB000C79AC5BC06BF07BF1093B80A1092BF0A66
:109DC0001092C60A1093C20A1092B90A1092C00AE1
:109DD000D092BC0A1092A5021092A6021092A00284
:109DE0001092A70A0E94E04F81E00E94134AEABE47
:109DF000F8BE89B7806F89BF0E9414590E948F4CAA
:109E00000E94E55678948DEE0E94F24F0E94F05821
:109E10000E9425510E947B5081E00E94AA4B0E9423
:109E20009B4A0E94B9580E949B558091A50283FFCE
:109E300007C0C098C09A80E00E94C0520E94294A80
:109E40000E9471588091A50287FFE0CF86CF8CE0F9
:109E50008093B80A8091A50284FF06C08E988091F5
:109E6000A5028F7E8093A50280E188BF14981C9A7A
:109E700008958CE08093C20A8091A50280FF06C0FD
:109E80008F988091A5028E7F8093A50280E288BF83
:109E900015981D9A08958823E9F477FF1BC065FD86
:109EA0001BC0CB0126E0969587952A95E1F7982F60
:109EB00092959F709827292F269526952927322F2E
:109EC0003695972F9295969596959370922793270E
:109ED00090FD03C080E0089580E00895282F22952A
:109EE0002F70282730E0A90156954795569547953C
:109EF000422753279A013695279524273527217025
:109F0000307020953095322F2227280F311D220FD7
:109F1000331F20503C4FC90108959091BE0A9F3FC6
:109F200011F19091BE0A9E3F21F49091C10A909345
:109F3000BE0AE091BE0AF0E0E855F54F80838091BB
:109F4000BE0A8F5F8093BE0A8091BE0A803110F0F6
:109F50001092BE0A9091BE0A8091C10A981719F416
:109F60008FEF8093BE0A08958091C10A8F3F21F13F
:109F70008091BE0A8031C0F49091BE0A8091C10ADE
:109F80009817D1F0E091C10AF0E0E855F54F8081D3
:109F90009091C10A9F5F9093C10A9091C10A90313C
:109FA00070F01092C10A08958091BE0A8E3F31F080
:109FB0009FEF9093C10A089580E0089580E008958E
:109FC0008FEF8093C10A08950E946E4F9093BB0A51
:109FD0008093BA0A8091A50280618093A5021C98A3
:109FE000149A08959091C60A992371F48093C60A31
:109FF0008D3E21F08F3F31F483E001C084E08093F7
:10A00000BF0A08951092C60A08951F93182F8A3F19
:10A0100009F46FC08E3F09F46CC08E3E09F469C02C
:10A020008A3A09F466C0813EE1F080912C018823D0
:10A03000C1F48091C10A8F3F29F48EEF8093BE0A4C
:10A040001092C10A8091BE0A8E3F41F480912F0187
:10A05000882339F480912E01882319F4812F0E94DE
:10A060008D4F80912C01882311F081500FC0103E3C
:10A0700021F481E080932E013CC0103F21F481E067
:10A0800080932F0136C0113E21F487E080932C018C
:10A0900030C080912D01181799F490912E01809174
:10A0A0001101981769F480912F01882331F01092E3
:10A0B0002D0181E08093110103C010922E0119C07F
:10A0C00040912F01442331F410932D0180912E01F2
:10A0D00080931101123121F480912E01882329F4FB
:10A0E000812F60912E010E94E94A10922E01109258
:10A0F0002F011F9108958091B80A8C3091F58091BD
:10A10000C60A882371F18091BF0A882351F184E146
:10A1100091E00197F1F700008091BF0A843021F4AB
:10A120008091C60A8D3E41F08091BF0A833039F498
:10A130008091C60A8F3F19F48091C60A0BC08091A6
:10A14000BF0A823071F48091C60A8D3E51F480912D
:10A15000A00287700E94E44F8091BF0A81508093D3
:10A16000BF0A8091B80A8C3060F48091C50A8823B8
:10A1700041F40E94274F1092BF0A1092C60A0E9413
:10A1800083498091B80A882309F050C08091A502C4
:10A1900084FD4AC08091B80A6091BA0A7091BB0AE6
:10A1A0000E944B4F9091C60A9923D1F19091C60A13
:10A1B0009D3E41F49091BF0A933061F09091BF0AA7
:10A1C000913041F09091C60A9F3FB9F49091BF0A37
:10A1D000923099F48A3F39F01092BF0A882341F0F7
:10A1E0000E94055005C08091BF0A81508093BF0A2C
:10A1F0008091BF0A8823C1F410C09091C60A9F3F86
:10A2000099F49091BF0A913079F48A3A21F0882329
:10A2100011F00E9405501092BF0A1092C60A04C0A5
:10A22000882311F00E9405500E94274F08950E9434
:10A230006E4F9093C40A8093C30A8091A5028160F7
:10A240008093A5021D98159A08951F938091C20AC4
:10A250008C3009F04DC0E091B90AF0E0EE5FFE4F9E
:10A260008081882391F08091C00A882309F040C042
:10A2700088E292E00197F1F700C00000E091B90A8E
:10A28000F0E0EE5FFE4F80812CC08091BC0A8823F5
:10A2900079F18091C00A882371F488E292E00197F5
:10A2A000F1F700C000008091A60281608093A602B1
:10A2B0008091BC0A16C08091A60280FF19C08091CF
:10A2C000BC0A883EA9F48091C00A823089F488E2F1
:10A2D00092E00197F1F700C000008DEF0E945956FF
:10A2E00083700E9417518091C00A8F5F8093C00ACB
:10A2F0008091C20A8C3098F48091BD0A882379F449
:10A300001091A5020E94394F10FF07C08091B90A31
:10A31000882319F40E94134A02C01092B90A80914E
:10A32000C20A882309F0F5C08091A50280FDEFC024
:10A330008091C20A6091C30A7091C40A0E944B4F77
:10A340009091A60290FF03C02091BC0A06C0E09144
:10A35000B90AF0E0EE5FFE4F208130E0283E310583
:10A3600009F493C0293E310524F42115310551F03B
:10A37000B3C0223F310509F45DC02F3F310509F01C
:10A38000ABC041C09091C00A9F5F9093C00A90916A
:10A39000C00A9230B1F0933020F4913009F0B7C088
:10A3A00006C09330A1F0943009F0B1C01FC02091D5
:10A3B000670197E098279F70207F920F9093670125
:10A3C000A6C090919F02980F90939F02A0C0909179
:10A3D0009D02980F90939D028091A50281FD97C0E8
:10A3E0001092C00A8091A50284604CC090916701D0
:10A3F0008295807F890F809367018091A502846098
:10A400008093A50282C09091C00A913011F48A3FD6
:10A41000F1F58091C00A8F5F8093C00A8091C00AD5
:10A42000843008F474C01092C00A8091A60280FFA4
:10A430004DC03CC09091C00A913041F49091C00A47
:10A440009F5F9093C00A8A3F11F561C01092C00AC5
:10A450009091A60290FF08C01092BC0A9091A602AB
:10A460009E7F9093A60205C09091B90A9F5F90933A
:10A47000B90A882321F08091A502826003C08091EF
:10A48000A5028D7F8093A50242C08A3F29F080916A
:10A49000A60280FF38C024C08091A60280FF14C0AD
:10A4A0008091C00A833050F01092C00A1092BC0A0A
:10A4B0008091A6028E7F8093A60229C08091C00A57
:10A4C0008F5F8093C00A23C01092C00A8091B90A9E
:10A4D0008F5F8093B90A1BC09091A60290FF08C0BD
:10A4E0001092BC0A8091A6028E7F8093A6020DC0B6
:10A4F0009091B90A9F5F9093B90A9091C00A9130E8
:10A5000021F48A3F11F01092B90A1092C00A0E94F9
:10A51000394F1F9108952091670130E0237030700A
:10A520002115310539F5893749F0893718F18B370D
:10A53000A1F08C37F9F48DEF60E009C08DEF0E9437
:10A540005956682F6370633009F06F5F8DEF0E947A
:10A550003E5688EE8093BC0A08958DEF0E945956AE
:10A56000682F637009F061508DEF0E943E5688EEAF
:10A570008093BC0A089580E78DB981E08EB9089573
:10A580008FB9779BFECF8FB108952091C70A309184
:10A59000C80AF901E955FD4F80832F5F3F4F37709F
:10A5A0003093C80A2093C70A2115310521F480E0B1
:10A5B00098E00E946F4E0895EF92FF921F93DF93F1
:10A5C000CF930F92CDB7DEB77C0110E00FC0E091C2
:10A5D000C70AF091C80AEE0DFF1DF770E955FD4F4F
:10A5E000808169830E94C5521F5F6981161778F3C5
:10A5F0000F90CF91DF911F91FF90EF900895B82FAA
:10A600009091C90A2091CA0AA0E001C0982F892F11
:10A6100081509923D1F42091A1023091A20240915E
:10A62000A3025091A402CA01B9016F5F7F4F8F4FFF
:10A630009F4F6093A1027093A2028093A302909314
:10A64000A4024BBFF901279187E0922F991F992708
:10A65000991FAA0FA92B220FB150C1F68093C90AE6
:10A660002093CA0A8A2F0895EF92FF920F931F93A7
:10A6700081E00E94FF52882341F184E00E94FF5252
:10A680002091A1023091A2024091A3025091A40214
:10A6900079018A010894E11CF11C011D111DE09251
:10A6A000A102F092A2020093A3021093A4024BBF56
:10A6B000F9012791806F482F50E041505040542FAE
:10A6C000442730E0422B532B1CC08091A102909173
:10A6D000A202A091A302B091A4029C01AD012F5F40
:10A6E0003F4F4F4F5F4F2093A1023093A202409300
:10A6F000A3025093A402ABBFFC018791482F50E006
:10A700005F6FCA011F910F91FF90EF9008950F9313
:10A710001F93CF93DF931092C80A1092C70A8091BB
:10A72000A1029091A202A091A302B091A4029C0167
:10A73000AD012F5F3F4F4F4F5F4F2093A1023093EA
:10A74000A2024093A3025093A402ABBFFC018791E5
:10A750000E94C5528091A1029091A202A091A302F1
:10A76000B091A4029C01AD012F5F3F4F4F4F5F4F4F
:10A770002093A1023093A2024093A3025093A4021B
:10A78000ABBFFC0187918093CA0A88E08093C90A15
:10A79000C1E0D0E081E00E94FF528823E1F0809187
:10A7A000A1029091A202A091A302B091A4029C01E7
:10A7B000AD012F5F3F4F4F4F5F4F2093A10230936A
:10A7C000A2024093A3025093A402ABBFFC01879165
:10A7D0000E94C552DFCF82E00E94FF52813079F0A3
:10A7E000813028F0823041F18330A1F629C083E026
:10A7F0000E94FF5290E0886F9F6F61E038C08091A7
:10A80000A1029091A202A091A302B091A4029C0186
:10A81000AD012F5F3F4F4F4F5F4F2093A102309309
:10A82000A2024093A3025093A402ABBFFC01879104
:10A8300090E09F6F62E01BC00E94345363E017C03A
:10A8400010E01F5F81E00E94FF528823D1F318308F
:10A85000A0F4812F0E94FF52082F0E943453BE01A2
:10A8600002C0660F771F1A95E2F76E5F600F0E94B5
:10A87000DC5290CF0E946F4E07C08091C70A909122
:10A88000C80A97700097B1F7DF91CF911F910F9190
:10A8900008951092980085E08093990010929B0093
:10A8A00088E180939A008EE080939D001092580179
:10A8B00081E0809357011092590180935D0180934C
:10A8C0005A011092560110925B0180E6809330018C
:10A8D00080EA809355018FEF80935C0110924301D1
:10A8E000109244011092420110923101089590910A
:10A8F0009B0095FFFCCF80939C000895EF92FF9200
:10A90000CF93DF93E82EE7017E01F92EE70102C025
:10A910000E94775489918823D9F7DF91CF91FF90D6
:10A92000EF9008958091580190915701292F282B7D
:10A9300009F187FF06C08F77809398009093990064
:10A940000895382F20E0290F311D40E050E060E0ED
:10A9500072EC81E090E00E94925960E07CE88AE02D
:10A9600090E00E947059215030403093980020931D
:10A97000990008951092980081E0809399000895BD
:10A9800080915601282F2770220F90E088739070D5
:10A990008830910521F08831910521F402C02063AF
:10A9A00001C0206220939D000895823009F43FC0C9
:10A9B000833030F4882371F0813009F066C02AC0FA
:10A9C000843009F456C0843008F44EC0873009F052
:10A9D0005CC059C08091560187FF03C06093570146
:10A9E0001FC08091420190913101891721F490910B
:10A9F000300195FF4AC0E82FF0E0EE5CFE4F608327
:10AA00008F5F8F7080934201809130018F798093A6
:10AA1000300108958091560187FF05C06093580169
:10AA20000E94925408956F70609359010895862F83
:10AA300060FF2BC061FF09C01092430110924401D6
:10AA4000909130019C7F9093300182FF09C0109259
:10AA50004201109231018091300180668093300173
:10AA6000697C60935D010895609356010E94C05413
:10AA70000895862F8F7180935B0161FF02C09598C6
:10AA80000895959A089560935C0108958330E1F1EB
:10AA9000843028F4813059F1823098F50AC085302D
:10AAA000C9F18530A0F18630C1F1873009F03FC08F
:10AAB0003BC08091560187FF03C0809157010895E4
:10AAC0002091300120FF35C090914401E92FF0E042
:10AAD000EB5BFE4F80819F5F9F70909344013091AC
:10AAE0004301931739F52E7F20933001089580910B
:10AAF000560187FF03C08091580108958091590144
:10AB0000089580915A010895809156010895809189
:10AB10005B01089580913001089580915501982F2F
:10AB2000907F90935501089580915C01089580E095
:10AB3000089580E008959091300195FD18C08091AE
:10AB40009B0085FF14C080913101E82FF0E0EE5C9E
:10AB5000FE4F208120939C008F5F8F708093310186
:10AB600020914201821719F49066909330018091F0
:10AB70009B0087FF1EC020919C0080914301909113
:10AB80004401891741F49091300190FF04C0926014
:10AB9000909330010EC0E82FF0E0EB5BFE4F208376
:10ABA0008F5F8F708093430180913001816080932B
:10ABB000300190919B008091300194FF02C0886029
:10ABC00001C0877F8093300190919B00809130017C
:10ABD00092FF02C0846001C08B7F8093300180911E
:10ABE0005501B69B09C084FF03C081608093550165
:10ABF000809155018F7E08C084FD03C081608093E1
:10AC0000550180915501806180935501089584EA32
:10AC1000809374008091740087FFFCCF8091710055
:10AC2000887F08958093730084E8809374008091F6
:10AC3000740087FFFCCF80917100887F0895809316
:10AC4000730084E8809374008091740087FFFCCFC8
:10AC500080917100887F0895982F92959F70990F29
:10AC6000292F220F220F290F8F70820F08956AE07B
:10AC70000E9464598295807F890F08950F931F93D6
:10AC8000182F062F0E940756887169F080EA0E94EB
:10AC90001256883141F4812F0E941F56883219F4D0
:10ACA000802F0E941F5684E9809374001F910F919A
:10ACB00008951F93182F0E9407568871F9F080EAB3
:10ACC0000E9412568831D1F4812F0E941F5688327B
:10ACD000A9F40E940756803189F481EA0E94125635
:10ACE000803461F484E8809374008091740087FF5D
:10ACF000FCCF809173009091710001C080E094E9D5
:10AD0000909374001F9108951F931092D50A82E0CA
:10AD10008093D60A1092D70A80E88093D80A86E0FA
:10AD20000E945956182F8F710E942C568093D30A77
:10AD3000129516951770173010F41F5F01C011E0BF
:10AD40001093D10A85E00E945956182F8F730E94E4
:10AD50002C568093D20A129516951695137010935F
:10AD6000D40A8FEF0E9459564091D40A282F30E020
:10AD70002370307050E04217530724F48C5F843600
:10AD800008F080E09091D40A8C7F890F8093D40AD8
:10AD90006091D40A8FEF0E943E5684E00E9459567B
:10ADA0008F730E942C568093CF0A83E00E945956DD
:10ADB0000E942C568093CD0A82E00E9459560E9430
:10ADC0002C568093CB0A1F9108951092710080E356
:10ADD000809370001092720080E060E00E943E5606
:10ADE0000E9484568091CB0A882311F40E948456D5
:10ADF0008EEF0E9459568B7F8093A00280E00E94C4
:10AE0000B74A08958091CB0A8F5F8093CB0A8091D7
:10AE1000CB0A8C3308F45CC01092CB0A8091CD0A27
:10AE20008F5F8093CD0A8091CD0A8C3308F450C097
:10AE30001092CD0A8091CF0A8F5F8093CF0A8091C4
:10AE4000CF0A883108F444C01092CF0A8091D10A09
:10AE50008F5F8093D10A8091D10A883018F081E009
:10AE60008093D10A8091D20A8F5F8093D20A309169
:10AE7000D20AE091D30AE150EC3008F0E0E0F0E0D3
:10AE8000EE5EFE4F20812C3141F48091D40A90E097
:10AE900083709070009709F42DE12317C8F491E0B6
:10AEA0009093D20A8091D30A8F5F8093D30A8091C6
:10AEB000D30A8D3068F09093D30A8091D40A8F5FC3
:10AEC0008093D40A8091D40A843610F01092D40A68
:10AED0008091D70A80618093D70A0895982F8E3089
:10AEE00008F5E82FF0E0E553F54F80819A3038F40B
:10AEF0009091D60A92FD1FC00E94375608959C304B
:10AF0000D1F49091D70A9F7E9093D70A26B330E070
:10AF10002095309520733070359527953595279578
:10AF2000822B0895803F20F08F700E94C8580895AA
:10AF30008E5F0E94595608951F93CF93DF93182F69
:10AF40008E3008F09CC08A3008F071C08091D60A1B
:10AF500082FD04C0862F0E942C56682FE12FF0E05E
:10AF6000E553F54F6083163071F1173038F4123025
:10AF7000B9F01430F1F0112351F08AC0183019F1F2
:10AF8000183008F445C0193009F082C03CC06C3359
:10AF900008F07EC0862F0E943756682F82E076C068
:10AFA0006C3308F075C0862F0E943756682F83E0F7
:10AFB0006DC0683108F06CC0862F0E943756682F2C
:10AFC0006F7384E063C08091D10A90E0883091056E
:10AFD0000CF05EC08091D30A882309F459C0809197
:10AFE000D30A8D3008F054C01091D10A8091D30A51
:10AFF0000E943756682F6F7111501295110F107EF5
:10B00000610F86E043C06091D40A8FEF0E943E56E4
:10B010001091D40A8091D20A0E943756682F6F731C
:10B020001295110F110F107C610F85E02FC08B302E
:10B0300019F08C3069F505C0647062606093D60ABF
:10B0400027C0C62FD0E0CE0180FF02C00E94E04F93
:10B050008091D70A90E08C279D2781FF19C08091AD
:10B06000D70A92E089278093D70A8091A00294E0C2
:10B0700089278093A0028DEE0E94F24F09C0803F85
:10B0800020F0862F0E94ED5803C08E5F0E943E562E
:10B09000DF91CF911F91089584B714BE009919C014
:10B0A00090E09C012E7130702115310511F080FF68
:10B0B00002C09F99FECF80916200886080936200F9
:10B0C00082E3EFEFF7ED3197F1F700C00000815018
:10B0D000C1F788EF809362001092DA0A1092D90AC1
:10B0E00008958091D90A9091DA0A26E0853A92076C
:10B0F00068F09F9906C080916200877F809362000C
:10B1000005C08091A50280688093A50280915E01B0
:10B1100090915F01009759F08091D90A9091DA0AD5
:10B12000009729F480E360E04FE70E94784A80911D
:10B13000D90A9091DA0A90935F0180935E01009999
:10B1400017C085B58F7C85BD9F9BFECF82E3EFEF57
:10B15000F7ED3197F1F700C000008150C1F7109270
:10B160005F0110925E018091A50280688093A50224
:10B1700008956091630060956F71809160018617FA
:10B1800031F06093600183E24FE70E94784A0895AE
:10B190008031F8F49091A70A913069F0913018F05D
:10B1A0009230C9F413C090E0A0E0B0E0805190422A
:10B1B000AE4FBF4F07C090E0A0E0B0E0805190409C
:10B1C000AE4FBF4FABBFFC01879108950E94B44FB3
:10B1D00008958FEF08958FEF08958093A70A08953B
:10B1E0001F93849B02C010E401C010E08091A5026F
:10B1F00090E080749070212F30E08217930791F0D7
:10B20000112311F084E001C080E00E94B74A1123AD
:10B2100021F08091A502806403C08091A5028F7BFC
:10B220008093A5021F910895E199FECF80E090E000
:10B230000E94AD598B3459F481E090E00E94AD59E1
:10B24000823429F48091A60282608093A602089538
:10B250001F938F3708F033C09091A60291FF0EC064
:10B26000882309F42CC080E092E00E94AD59182F89
:10B2700081E092E00E94AD59982F23C090E0880FA2
:10B28000991FAA2797FDA095BA2F662329F02CE8CD
:10B2900031E040E0552704C02CE830E040E055277D
:10B2A000280F391F4A1F5B1F4BBFF90117912F5FF2
:10B2B0003F4F4F4F5F4F4BBFF901979102C09FE740
:10B2C0001FE7812F1F910895991B79E004C0991FF2
:10B2D000961708F0961B881F7A95C9F780950895F0
:10B2E000A1E21A2EAA1BBB1BFD010DC0AA1FBB1F8A
:10B2F000EE1FFF1FA217B307E407F50720F0A21BFC
:10B30000B30BE40BF50B661F771F881F991F1A9468
:10B3100069F760957095809590959B01AC01BD0192
:10B32000CF01089597FB092E05260ED057FD04D0B6
:10B33000D7DF0AD0001C38F4509540953095219500
:10B340003F4F4F4F5F4F0895F6F79095809570955A
:10B3500061957F4F8F4F9F4F0895E199FECF9FBB1F
:0EB360008EBBE09A99278DB30895F894FFCF25
:10B36E00FF01FFFFFFF3C8F364F350F2E6F364F45A
:10B37E0000011F1C1F1E1F1E1F1F1E1F1E1FF0DF82
:06B38E000100F0FF0100C8
:00000001FF
